:020000040000FA
:0408000039EF08F0D4
:1008100003B213EF05F0F2B42EEF05F09EB036EF01
:1008200005F09EB23EEF05F0F2A81AEF04F0F2B226
:1008300025EF04F0F2A620EF04F0F2B022EF04F06E
:10084000E8EF07F0F296F290FF00CD90F2929EA0B2
:100850002FEF04F00101533F2FEF04F0542BAEC1F2
:10086000B2F1AFC1B3F1B0C1B4F1B1C1B5F1AAC138
:10087000AEF1ABC1AFF1ACC1B0F1ADC1B1F1A6C148
:10088000AAF1A7C1ABF1A8C1ACF1A9C1ADF1A2C158
:10089000A6F1A3C1A7F1A4C1A8F1A5C1A9F19EC168
:1008A000A2F19FC1A3F1A0C1A4F1A1C1A5F19AC178
:1008B0009EF19BC19FF19CC1A0F19DC1A1F196C188
:1008C0009AF197C19BF198C19CF199C19DF1CECF4E
:1008D00096F1CFCF97F153C198F154C199F1CF6AF6
:1008E000CE6A0101536B546B9E90CD800FBC0F8E6E
:1008F0000FBA7EEF04F00F8AE8EF07F00F8C0FBEFF
:10090000BAEF04F096C19AF197C19BF198C19CF19E
:1009100099C19DF19AC19EF19BC19FF19CC1A0F12B
:100920009DC1A1F19EC1A2F19FC1A3F1A0C1A4F1FB
:10093000A1C1A5F1A2C1A6F1A3C1A7F1A4C1A8F1CB
:10094000A5C1A9F1A6C1AAF1A7C1ABF1A8C1ACF19B
:10095000A9C1ADF1AAC1AEF1ABC1AFF1ACC1B0F16B
:10096000ADC1B1F1AEC1B2F1AFC1B3F1B0C1B4F13B
:10097000B1C1B5F101015E6B5F6B606B616B96514C
:100980005E2797515F2398516023995161239A51B3
:100990005E279B515F239C5160239D5161239E5193
:1009A0005E279F515F23A0516023A1516123A25173
:1009B0005E27A3515F23A4516023A5516123A65153
:1009C0005E27A7515F23A8516023A9516123AA5133
:1009D0005E27AB515F23AC516023AD516123AE5113
:1009E0005E27AF515F23B0516023B1516123B251F3
:1009F0005E27B3515F23B4516023B5516123D89072
:100A00000101613360335F335E33D890010161339C
:100A100060335F335E33D8900101613360335F33FD
:100A20005E33E8EF07F00392030103EE00F080511C
:100A30007F0BE92604C0EFFF802B8151805D700B96
:100A4000D8A48B8200008051815D700BD8A48B925A
:100A500081518019D8B40790E8EF07F0F2940101B2
:100A6000453FE8EF07F0462BE8EF07F09E900101C5
:100A7000533FE8EF07F0542BE8EF07F09E92040095
:100A800062A143EF05F007B495EF05F007B095EFCD
:100A900005F01EC620F61FC621F61CC61EF61DC692
:100AA0001FF61AC61CF61BC61DF606C608F607C6B4
:100AB00009F604C606F605C607F602C604F603C61E
:100AC00005F626C628F627C629F624C626F625C624
:100AD00027F622C624F623C625F60EC610F60FC644
:100AE00011F60CC60EF60DC60FF60AC60CF60BC6AE
:100AF0000DF62EC630F62FC631F62CC62EF62DC6B4
:100B00002FF62AC62CF62BC62DF616C618F617C6D3
:100B100019F614C616F615C617F612C614F613C63D
:100B200015F6AAEC2AF042EC2AF0077C07ACB0EFED
:100B300005F0C274C2B4AAEF05F0C3CFB3F5C4CFB9
:100B4000B4F50501D890B433B333D890B433B3338C
:100B5000B1EF05F0C3CF55F1C4CF56F1B1EF05F0B9
:100B6000C28207B41EEF06F047C14BF148C14CF1F9
:100B700049C14DF14AC14EF15EC162F15FC163F1FD
:100B800060C164F161C165F196C1B6F197C1B7F179
:100B900098C1B8F199C1B9F19AC1BAF19BC1BBF141
:100BA0009CC1BCF19DC1BDF19EC1BEF19FC1BFF111
:100BB000A0C1C0F1A1C1C1F1A2C1C2F1A3C1C3F1E1
:100BC000A4C1C4F1A5C1C5F1A6C1C6F1A7C1C7F1B1
:100BD000A8C1C8F1A9C1C9F1AAC1CAF1ABC1CBF181
:100BE000ACC1CCF1ADC1CDF1AEC1CEF1AFC1CFF151
:100BF000B0C1D0F1B1C1D1F1B2C1D2F1B3C1D3F121
:100C0000B4C1D4F1B5C1D5F1B3C5B5F5B4C5B6F528
:100C1000B5C5B7F5B6C5B8F5010155515B275651B5
:100C20005C23E86A5D230E2E1EEF06F05CC157F1CF
:100C30005DC158F15B6B5C6B5D6B078E0201002F31
:100C4000E8EF07F03C0E006F00C10CF101C10DF19F
:100C500002C10EF103C10FF104C110F105C111F180
:100C600006C112F107C113F108C114F109C115F150
:100C70000AC116F10BC117F134C135F105012F512D
:100C8000000AD8B4E7EF06F005012F51010AD8B4E5
:100C900071EF06F005012F51020AD8B4B2EF06F049
:100CA00005012F51030AD8B4B2EF06F005012F5108
:100CB000040AD8B4B2EF06F005012F51050AD8B4E2
:100CC000B2EF06F005012F51060AD8B4B2EF06F0D4
:100CD00005012F51070AD8B4B2EF06F02F6BE7EFEA
:100CE00006F0050153677CEF06F054677CEF06F0D1
:100CF00055677CEF06F0566780EF06F0E7EF06F0E9
:100D000057C500F158C501F159C502F15AC503F1A3
:100D10000101010E046F000E056F000E066F000E3C
:100D2000076FB3EC28F000C157F501C158F502C1B7
:100D300059F503C15AF50067A5EF06F00167A5EF65
:100D400006F00267A5EF06F00367E7EF06F053C56C
:100D500057F554C558F555C559F556C55AF50F8878
:100D6000E7EF06F005013067B8EF06F0E7EF06F0B1
:100D70000FBECDEF06F010A0D2EF06F001014767DD
:100D8000C9EF06F04867C9EF06F04967C9EF06F0FA
:100D90004A67CDEF06F0D2EF06F007AED2EF06F0CD
:100DA000E4EF06F00501312FE7EF06F03C0E316F5E
:100DB000302FE7EF06F00101000E626FE00E636F67
:100DC000A50E646F010E656F0501306B0F8805017C
:100DD000626B33B7EDEF06F062810CC100F10DC11B
:100DE00001F10EC102F10FC103F110C104F111C1F3
:100DF00005F112C106F113C107F114C108F115C1C3
:100E000009F116C10AF117C10BF135C134F100C166
:100E10000CF101C10DF102C10EF103C10FF104C1CA
:100E200010F105C111F106C112F107C113F108C19A
:100E300014F109C115F10AC116F10BC117F134C142
:100E400035F101018A672CEF07F08B672CEF07F073
:100E50008C672CEF07F08D6730EF07F060EF07F03D
:100E60008EC100F18FC101F190C102F191C103F176
:100E70000101010E046F000E056F000E066F000EDB
:100E8000076FB3EC28F000C18EF101C18FF102C1F0
:100E900090F103C191F1006755EF07F0016755EF3D
:100EA00007F0026755EF07F0036760EF07F08AC1AC
:100EB0008EF18BC18FF18CC190F18DC191F10F80BA
:100EC000D57ED5BE69D0D6CF47F1D7CF48F145C141
:100ED00049F1E86AE8CF4AF1109047C100F148C1F2
:100EE00001F149C102F14AC103F101010A0E046F87
:100EF000000E056F000E066F000E076FB3EC28F0B2
:100F000003AF1080010154A792EF07F00F9A0F9CD6
:100F10000F9E0101000E5E6F600E5F6F3D0E606FF1
:100F2000080E616F010147BFA2EF07F04867A2EF0B
:100F300007F04967A2EF07F04A67A2EF07F0F288CF
:100F4000C7EF07F0F2985E6B5F6B606B616B966B3F
:100F5000976B986B996B9A6B9B6B9C6B9D6B9E6B65
:100F60009F6BA06BA16BA26BA36BA46BA56BA66B15
:100F7000A76BA86BA96BAA6BAB6BAC6BAD6BAE6BC5
:100F8000AF6BB06BB16BB26BB36BB46BB56BD76A55
:100F9000D66A0101456B466B0CC100F10DC101F130
:100FA0000EC102F10FC103F110C104F111C105F12D
:100FB00012C106F113C107F114C108F115C109F1FD
:100FC00016C10AF117C10BF135C134F1E8EF07F092
:100FD00002C0E0FF005001C0D8FF1000A6B2EEEF43
:100FE00007F00CC0A9FF0BC0A8FFA69EA69CA68474
:100FF000F29E550EA76EAA0EA76EA682F28EA6943A
:10100000A6B200EF08F00C2A1200A96EA69EA69CBC
:10101000A680A8500C2A120004012C0E826F29EC25
:101020000BF0AEEC29F00C5005EC08F0E8CF00F125
:101030000C5005EC08F0E8CF01F101AF25EF08F006
:101040000101FF0E026FFF0E036F51EC29F02967BB
:1010500031EF08F00401200E826F29EC0BF036EF1F
:1010600008F004012D0E826F29EC0BF07BEC27F0C9
:101070001200076A0F6A106A0F010D0EC16E860E0C
:10108000C06E030EC26E0F01680E896E130E926E53
:10109000080E8A6E8A6AF30E936E8B6A900E946EB7
:1010A000F18EF19E0E6A01015B6B5C6B5D6B576BA1
:1010B000586BF29A0101476B486B496B4A6B4B6B5B
:1010C0004C6B4D6B4E6B4F6B506B516B526B456B5A
:1010D000466BD76AD66A0F01280ED56EF28A9D90AC
:1010E000B00ECD6E01015E6B5F6B606B616B626B0E
:1010F000636B646B656B666B676B686B696B536B7B
:10110000546BCF6ACE6A0F9A0F9C0F9E9D80760E0D
:10111000CA6E9D8202013C0E006FCC6A160E05EC71
:1011200008F0E8CF00F1170E05EC08F0E8CF01F168
:10113000180E05EC08F0E8CF02F1190E05EC08F0E6
:10114000E8CF03F1010103AFC0EF08F0AEEC29F0E6
:10115000160E0C6E00C10BF0EEEC07F0170E0C6EC5
:1011600001C10BF0EEEC07F0180E0C6E02C10BF093
:10117000EEEC07F0190E0C6E03C10BF0EEEC07F06D
:1011800000C18AF101C18BF102C18CF103C18DF163
:1011900000C18EF101C18FF102C190F103C191F143
:1011A0001A0E05EC08F0E8CF00F11B0E05EC08F074
:1011B000E8CF01F11C0E05EC08F0E8CF02F11D0E9E
:1011C00005EC08F0E8CF03F1010103AF16EF09F0D9
:1011D000AEEC29F01A0E0C6E00C10BF0EEEC07F02D
:1011E0001B0E0C6E01C10BF0EEEC07F01C0E0C6E2A
:1011F00002C10BF0EEEC07F01D0E0C6E03C10BF0FC
:10120000EEEC07F01A0E05EC08F0E8CF00F11B0E2B
:1012100005EC08F0E8CF01F11C0E05EC08F0E8CF72
:1012200002F11D0E05EC08F0E8CF03F100C192F1C8
:1012300001C193F102C194F103C195F1240EAC6E8A
:10124000900EAB6E240EAC6E080EB86E000EB06E33
:101250001F0EAF6E0401806B816B0F01900EAB6EA1
:101260000F019D8A0301806B816BC26B8B923DECF9
:1012700030F03DEC30F0880E05EC08F0E8CF00F1DE
:10128000890E05EC08F0E8CF01F1010101AF61EF33
:1012900009F0AEEC29F0880E0C6E00C10BF0EEECFC
:1012A00007F0890E0C6E01C10BF0EEEC07F0880E12
:1012B00005EC08F0E8CF00F1890E05EC08F0E8CF66
:1012C00001F100C140F601C141F602C142F603C17D
:1012D00043F693EC33F01EEC2EF0200E05EC08F0F4
:1012E000E8CF2FF505012F51FF0AD8A47FEF09F0B1
:1012F0002F6B200E0C6E2FC50BF0EEEC07F00501E6
:10130000010E306F3C0E316F250E05EC08F0E8CF72
:1013100000F1260E05EC08F0E8CF01F1270E05ECF0
:1013200008F0E8CF02F1280E05EC08F0E8CF03F151
:10133000010103AFB6EF09F0AEEC29F0250E0C6EFB
:1013400000C10BF0EEEC07F0260E0C6E01C10BF0A5
:10135000EEEC07F0270E0C6E02C10BF0EEEC07F07E
:10136000280E0C6E03C10BF0EEEC07F000C153F534
:1013700001C154F502C155F503C156F500C157F539
:1013800001C158F502C159F503C15AF5290E05EC02
:1013900008F0E8CF5BF505015C515B5DD8A05BC54B
:1013A0005CF505012F51020A0EE181B8E3EF09F067
:1013B00005015C2FE0EF09F05BC55CF5E3EF09F098
:1013C00081BAD2EF33F0210E05EC08F0E8CF00F13E
:1013D000220E05EC08F0E8CF01F1230E05EC08F031
:1013E000E8CF02F1240E05EC08F0E8CF03F101018B
:1013F00003AF29EF0AF0AEEC29F0210E0C6E00C10C
:101400000BF0EEEC07F0220E0C6E01C10BF0EEECCF
:1014100007F0230E0C6E02C10BF0EEEC07F0240E69
:101420000C6E03C10BF0EEEC07F0210E05EC08F09A
:10143000E8CF00F1220E05EC08F0E8CF01F1230E11
:1014400005EC08F0E8CF02F1240E05EC08F0E8CF37
:1014500003F100C15DF501C15EF502C15FF503C195
:1014600060F555EC2DF017EC2CF067EC2BF0050136
:101470002F51030A12E005012F51040A1DE0050156
:101480002F51050A24E005012F51060A32E005011B
:101490002F51070A38E08CEF0AF0ACC500F10101CA
:1014A0000F0E001701010051000A36E00101005142
:1014B000050A32E089EF0AF0ACC500F101010F0E18
:1014C000001701010051000A27E089EF0AF0050129
:1014D000AC51000A21E00501AC51150A1DE00501DF
:1014E000AC51300A19E00501AC51450A15E089EF0D
:1014F0000AF00501AC51000A0FE00501AC51300AB9
:101500000BE089EF0AF00501AC51000A05E089EF14
:101510000AF081BAD2EF33F012EC2BF00790000101
:10152000F28EF28C07B00FEF25F00FB0F0EF1FF046
:101530000FB8B4EF19F00301805181197F0BD8B4B3
:101540000FEF25F013EE00F081517F0BE126812B88
:10155000E7CFE8FFE00BD8B40FEF25F023EE82F0E1
:10156000C2513F0BD926E7CFDFFFC22BDF50780AED
:10157000D8A40FEF25F007808EC100F18FC101F1D3
:1015800090C102F191C103F10101040E046F000E3C
:10159000056F000E066F000E076FB3EC28F000AF6A
:1015A000DBEF0AF00101030E8E6F000E8F6F000E4D
:1015B000906F000E916F03018251720AD8B4F0EF60
:1015C0001FF08251520AD8B4F0EF1FF08251750A11
:1015D000D8B4F0EF1FF08251630AD8B4CBEF21F0FA
:1015E0008251690AD8B4ABEF1CF082517A0AD8B4A0
:1015F000BEEF1DF08251490AD8B44AEF1CF0825167
:10160000500AD8B468EF1BF08251700AD8B4ABEF1F
:101610001BF08251540AD8B4D6EF1BF08251740AE1
:10162000D8B41CEF1CF08251730AD8B420EF1FF01D
:101630008251530AD8B485EF1FF082514C0AD8B4B6
:1016400016EF12F08251760AD8B43DEF0BF000EF9E
:1016500022F0040114EE00F080517F0BE12682C4D9
:10166000E7FF802B120004010D0E826F29EC0BF0B6
:101670000A0E826F29EC0BF0120003018351300A2D
:10168000D8B4E7EF0CF003018351310AD8B41EEF50
:101690000DF003018351320AD8B4D3EF0EF00301E9
:1016A0008351330AD8B488EF10F003018351340A10
:1016B000D8B42EEF11F003018351730AD8B4C4EFEC
:1016C0000BF003018351760AD8B4C6EF0BF0030187
:1016D0008351740AD8B4B1EF0BF003018351540A5B
:1016E000D8B476EF0BF0D8A400EF22F00401560E28
:1016F000826F29EC0BF00401540E826F29EC0BF081
:1017000007840001880E0C6EEFEC29F0298103019B
:1017100084512D0AD8B48FEF0BF00101299185C3B4
:101720002FF186C330F187C331F188C332F189C309
:1017300033F1FCEC29F073EC29F000C10BF0EEEC76
:1017400007F001C10BF0EEEC07F0880E05EC08F095
:10175000E8CF40F6890E05EC08F0E8CF41F6BCEF83
:101760000BF00401560E826F29EC0BF00401740E8D
:10177000826F29EC0BF007840001880E0C6E0CECD4
:1017800008F0079415EF1AF0C4EC0BF00401760E84
:10179000826F29EC0BF00401760E826F29EC0BF0BE
:1017A00004012C0E826F29EC0BF007842BEC26F041
:1017B00004012C0E826F29EC0BF00101036B026B0C
:1017C0003BC601F13AC600F101AFECEF0BF00101AD
:1017D000FF0E026FFF0E036F51EC29F02967F3EF44
:1017E0000BF0F8EF0BF004012D0E826F29EC0BF0DB
:1017F0002FC182F40401300E822729EC0BF030C196
:1018000082F40401300E822729EC0BF031C182F4FE
:101810000401300E822729EC0BF032C182F404015E
:10182000300E822729EC0BF033C182F40401300E14
:10183000822729EC0BF004012C0E826F29EC0BF0AF
:101840000101036B026B3DC601F13CC600F101AF23
:101850002FEF0CF00101FF0E026FFF0E036F51EC32
:1018600029F0296736EF0CF03BEF0CF004012D0E48
:10187000826F29EC0BF02FC182F40401300E822715
:1018800029EC0BF030C182F40401300E822729ECE0
:101890000BF031C182F40401300E822729EC0BF0E9
:1018A00032C182F40401300E822729EC0BF033C1DF
:1018B00082F40401300E822729EC0BF004012C0E77
:1018C000826F29EC0BF00101036B026B3FC601F143
:1018D0003EC600F101AF72EF0CF00101FF0E026F86
:1018E000FF0E036F51EC29F0296779EF0CF07EEFC2
:1018F0000CF004012D0E826F29EC0BF02FC182F445
:101900000401300E822729EC0BF030C182F404016F
:10191000300E822729EC0BF031C182F40401300E25
:10192000822729EC0BF032C182F40401300E8227A9
:1019300029EC0BF033C182F40401300E822729EC2C
:101940000BF004012C0E826F29EC0BF00101036BEC
:10195000026B37C601F136C600F101AFB5EF0CF0EE
:101960000101FF0E026FFF0E036F51EC29F0296792
:10197000BCEF0CF0C1EF0CF004012D0E826F29ECCE
:101980000BF02FC182F40401300E822729EC0BF0FA
:1019900030C182F40401300E822729EC0BF031C1F2
:1019A00082F40401300E822729EC0BF032C182F45C
:1019B0000401300E822729EC0BF033C182F40401BC
:1019C000300E822729EC0BF0079415EF1AF0040172
:1019D000760E826F29EC0BF00401300E826F29EC39
:1019E0000BF004012C0E826F29EC0BF01CEC2AF09A
:1019F000AEEC29F000C600F101C601F151EC29F06E
:101A000030C182F40401300E822729EC0BF031C181
:101A100082F40401300E822729EC0BF032C182F4EB
:101A20000401300E822729EC0BF033C182F404014B
:101A3000300E822729EC0BF015EF1AF00401760E18
:101A4000826F29EC0BF00401310E826F29EC0BF050
:101A500007840101036B026B02C600F103C601F1AA
:101A600001AF37EF0DF0FF0E026FFF0E036F0101A4
:101A7000076B066B04C604F105C605F105AF45EF1B
:101A80000DF0FF0E066FFF0E076FB8EC28F0010196
:101A9000076B066B06C604F107C605F105AF55EFE7
:101AA0000DF0FF0E066FFF0E076FB8EC28F0010176
:101AB000076B066B08C604F109C605F105AF65EFB3
:101AC0000DF0FF0E066FFF0E076FB8EC28F0D890F0
:101AD00001010333023301330033D8900101033392
:101AE00002330133003304012C0E826F29EC0BF01A
:101AF0000101036B026B01C101F100C100F101AFF3
:101B000087EF0DF00101FF0E026FFF0E036F51EC26
:101B100029F029678EEF0DF093EF0DF004012D0EE3
:101B2000826F29EC0BF02FC182F40401300E822762
:101B300029EC0BF030C182F40401300E822729EC2D
:101B40000BF031C182F40401300E822729EC0BF036
:101B500032C182F40401300E822729EC0BF033C12C
:101B600082F40401300E822729EC0BF00101036B93
:101B7000026B0AC600F10BC601F101AFC4EF0DF014
:101B8000FF0E026FFF0E036F0101076B066B0CC6A1
:101B900004F10DC605F105AFD2EF0DF0FF0E066F93
:101BA000FF0E076FB8EC28F00101076B066B0EC63D
:101BB00004F10FC605F105AFE2EF0DF0FF0E066F61
:101BC000FF0E076FB8EC28F00101076B066B10C61B
:101BD00004F111C605F105AFF2EF0DF0FF0E066F2F
:101BE000FF0E076FB8EC28F0D890010103330233E1
:101BF00001330033D8900101033302330133003342
:101C000004012C0E826F29EC0BF00101036B026BB7
:101C100001C101F100C100F101AF14EF0EF00101AB
:101C2000FF0E026FFF0E036F51EC29F029671BEFC7
:101C30000EF020EF0EF004012D0E826F29EC0BF058
:101C40002FC182F40401300E822729EC0BF030C141
:101C500082F40401300E822729EC0BF031C182F4AA
:101C60000401300E822729EC0BF032C182F404010A
:101C7000300E822729EC0BF033C182F40401300EC0
:101C8000822729EC0BF00101036B026B12C600F1F5
:101C900013C601F101AF51EF0EF0FF0E026FFF0E00
:101CA000036F0101076B066B14C604F115C605F13D
:101CB00005AF5FEF0EF0FF0E066FFF0E076FB8EC7B
:101CC00028F00101076B066B16C604F117C605F173
:101CD00005AF6FEF0EF0FF0E066FFF0E076FB8EC4B
:101CE00028F00101076B066B18C604F119C605F14F
:101CF00005AF7FEF0EF0FF0E066FFF0E076FB8EC1B
:101D000028F0D89001010333023301330033D89017
:101D10000101033302330133003304012C0E826FBF
:101D200029EC0BF00101036B026B01C101F100C151
:101D300000F101AFA1EF0EF00101FF0E026FFF0EE7
:101D4000036F51EC29F02967A8EF0EF0ADEF0EF00C
:101D500004012D0E826F29EC0BF02FC182F40401D7
:101D6000300E822729EC0BF030C182F40401300ED2
:101D7000822729EC0BF031C182F40401300E822756
:101D800029EC0BF032C182F40401300E822729ECD9
:101D90000BF033C182F40401300E822729EC0BF0E2
:101DA000079415EF1AF00401760E826F29EC0BF000
:101DB0000401320E826F29EC0BF007840101036BE2
:101DC000026B1AC600F11BC601F101AFECEF0EF079
:101DD000FF0E026FFF0E036F0101076B066B1CC63F
:101DE00004F11DC605F105AFFAEF0EF0FF0E066F08
:101DF000FF0E076FB8EC28F00101076B066B1EC6DB
:101E000004F11FC605F105AF0AEF0FF0FF0E066FD4
:101E1000FF0E076FB8EC28F00101076B066B20C6B8
:101E200004F121C605F105AF1AEF0FF0FF0E066FA2
:101E3000FF0E076FB8EC28F0D8900101033302338E
:101E400001330033D89001010333023301330033EF
:101E500004012C0E826F29EC0BF00101036B026B65
:101E600001C101F100C100F101AF3CEF0FF0010130
:101E7000FF0E026FFF0E036F51EC29F0296743EF4D
:101E80000FF048EF0FF004012D0E826F29EC0BF0DC
:101E90002FC182F40401300E822729EC0BF030C1EF
:101EA00082F40401300E822729EC0BF031C182F458
:101EB0000401300E822729EC0BF032C182F40401B8
:101EC000300E822729EC0BF033C182F40401300E6E
:101ED000822729EC0BF00101036B026B22C600F193
:101EE00023C601F101AF79EF0FF0FF0E026FFF0E75
:101EF000036F0101076B066B24C604F125C605F1CB
:101F000005AF87EF0FF0FF0E066FFF0E076FB8ECFF
:101F100028F00101076B066B26C604F127C605F100
:101F200005AF97EF0FF0FF0E066FFF0E076FB8ECCF
:101F300028F00101076B066B28C604F129C605F1DC
:101F400005AFA7EF0FF0FF0E066FFF0E076FB8EC9F
:101F500028F0D89001010333023301330033D890C5
:101F60000101033302330133003304012C0E826F6D
:101F700029EC0BF00101036B026B01C101F100C1FF
:101F800000F101AFC9EF0FF00101FF0E026FFF0E6C
:101F9000036F51EC29F02967D0EF0FF0D5EF0FF068
:101FA00004012D0E826F29EC0BF02FC182F4040185
:101FB000300E822729EC0BF030C182F40401300E80
:101FC000822729EC0BF031C182F40401300E822704
:101FD00029EC0BF032C182F40401300E822729EC87
:101FE0000BF033C182F40401300E822729EC0BF090
:101FF0000101036B026B2AC600F12BC601F101AF90
:1020000006EF10F0FF0E026FFF0E036F0101076B6A
:10201000066B2CC604F12DC605F105AF14EF10F0C8
:10202000FF0E066FFF0E076FB8EC28F00101076B7B
:10203000066B2EC604F12FC605F105AF24EF10F094
:10204000FF0E066FFF0E076FB8EC28F00101076B5B
:10205000066B30C604F131C605F105AF34EF10F060
:10206000FF0E066FFF0E076FB8EC28F0D890010145
:102070000333023301330033D890010103330233B9
:102080000133003304012C0E826F29EC0BF00101A7
:10209000036B026B01C101F100C100F101AF56EF0A
:1020A00010F00101FF0E026FFF0E036F51EC29F0DB
:1020B00029675DEF10F062EF10F004012D0E826FC2
:1020C00029EC0BF02FC182F40401300E822729EC99
:1020D0000BF030C182F40401300E822729EC0BF0A2
:1020E00031C182F40401300E822729EC0BF032C199
:1020F00082F40401300E822729EC0BF033C182F404
:102100000401300E822729EC0BF0079415EF1AF02A
:102110000401760E826F29EC0BF00401330E826FFE
:1021200029EC0BF004012C0E826F29EC0BF085C317
:1021300082F429EC0BF0640E0D6E03018551320A16
:1021400002E16A0E0D6E03018551330A02E1700E41
:102150000D6E03018551340A02E1760E0D6E030106
:102160008551350A02E17C0E0D6E03018551360A58
:1021700002E1820E0D6E03018651780A65E00DC002
:102180000CF0EFEC29F02981030187512D0AD8B416
:10219000CCEF10F00101299188C32FF189C330F1F0
:1021A0008AC331F18BC332F18CC333F1FCEC29F0DB
:1021B00073EC29F000C10BF0EEEC07F001C10BF05D
:1021C000EEEC07F0EFEC29F0298103018E512D0A86
:1021D000D8B4EDEF10F0010129918FC32FF190C316
:1021E00030F191C331F192C332F193C333F1FCEC7E
:1021F00029F073EC29F000C10BF0EEEC07F001C1FF
:102200000BF0EEEC07F0EFEC29F02981030195517A
:102210002D0AD8B40EEF11F00101299196C32FF1C8
:1022200097C330F198C331F199C332F19AC333F1B6
:10223000FCEC29F073EC29F000C10BF0EEEC07F098
:1022400001C10BF0EEEC07F00DC00CF00CEC08F047
:102250000CEC08F00CEC08F015EF1AF00401760E07
:10226000826F29EC0BF00401340E826F29EC0BF025
:1022700003018451780AD8B406EF12F03E0E0C6EBA
:10228000EFEC29F02981030185512D0AD8B44BEFD9
:1022900011F00101299186C32FF187C330F188C362
:1022A00031F189C332F18AC333F1FCEC29F073ECCC
:1022B00029F000C10BF0EEEC07F001C10BF0EEECE1
:1022C00007F0EFEC29F0298103018C512D0AD8B4D5
:1022D0006CEF11F0010129918DC32FF18EC330F104
:1022E0008FC331F190C332F191C333F1FCEC29F08B
:1022F00073EC29F000C10BF0EEEC07F001C10BF01C
:10230000EEEC07F0EFEC29F02981030193512D0A3F
:10231000D8B48DEF11F00101299194C32FF195C329
:1023200030F196C331F197C332F198C333F1FCEC2D
:1023300029F073EC29F000C10BF0EEEC07F001C1BD
:102340000BF0EEEC07F0EFEC29F0298103019A5134
:102350002D0AD8B4AEEF11F0010129919BC32FF1E2
:102360009CC330F19DC331F19EC332F19FC333F161
:10237000FCEC29F073EC29F000C10BF0EEEC07F057
:1023800001C10BF0EEEC07F0EFEC29F0298103011D
:10239000A1512D0AD8B4CFEF11F001012991A2C3A8
:1023A0002FF1A3C330F1A4C331F1A5C332F1A6C309
:1023B00033F1FCEC29F073EC29F000C10BF0EEECEA
:1023C00007F001C10BF0EEEC07F0EFEC29F02981EA
:1023D0000301A8512D0AD8B4F0EF11F001012991A1
:1023E000A9C32FF1AAC330F1ABC331F1ACC332F1B1
:1023F000ADC333F1FCEC29F073EC29F000C10BF014
:10240000EEEC07F001C10BF0EEEC07F03E0E0C6EA7
:102410000CEC08F00CEC08F00CEC08F00CEC08F0FC
:102420000CEC08F00CEC08F015EF1AF003018351E6
:10243000300AD8B4D7EF14F003018351310AD8B46D
:10244000E5EF15F003018351320AD8B453EF16F0CB
:1024500003018351330AD8B463EF16F003018351AB
:10246000340AD8B473EF16F003018351350AD8B497
:10247000B9EF19F003018351360AD8B4E7EF19F028
:1024800003018351460AD8B40DEF19F003018351BB
:102490004D0AD8B450EF13F0030183516D0AD8B43C
:1024A0006AEF13F0030183515A0AD8B45FEF15F0B5
:1024B00003018351490AD8B4E7EF1AF003018351AD
:1024C000500AD8B419EF1AF003018351540AD8B452
:1024D00092EF1AF003018351630AD8B48AEF13F024
:1024E00003018351430AD8B482EF14F003018351EE
:1024F000730AD8B488EF13F003018351610AD8B48A
:102500009DEF12F003018351650AD8B427EF15F04F
:1025100003018351450AD8B435EF15F00301835107
:10252000620AD8B443EF15F003018351420AD8B4CC
:1025300051EF15F0D8A400EF22F004014C0E826F89
:1025400029EC0BF00401610E826F29EC0BF017EC03
:102550002CF004012C0E826F29EC0BF0AEEC29F06C
:10256000ABC500F1010151EC29F031C182F4040145
:10257000300E822729EC0BF032C182F40401300EB8
:10258000822729EC0BF033C182F40401300E82273C
:1025900029EC0BF004012C0E826F29EC0BF0AEEC51
:1025A00029F0ACC500F1010151EC29F031C182F4F0
:1025B0000401300E822729EC0BF032C182F40401B1
:1025C000300E822729EC0BF033C182F40401300E67
:1025D000822729EC0BF004012C0E826F29EC0BF002
:1025E000AEEC29F0ADC500F1010151EC29F031C18B
:1025F00082F40401300E822729EC0BF032C182F400
:102600000401300E822729EC0BF033C182F404015F
:10261000300E822729EC0BF004012C0E826F29EC7E
:102620000BF0AEEC29F0AEC500F1010151EC29F040
:1026300031C182F40401300E822729EC0BF032C143
:1026400082F40401300E822729EC0BF033C182F4AE
:102650000401300E822729EC0BF004012C0E826F4E
:1026600029EC0BF0AEEC29F0B3C500F1010151ECFF
:1026700029F031C182F40401300E822729EC0BF0DD
:1026800032C182F40401300E822729EC0BF033C1F1
:1026900082F40401300E822729EC0BF015EF1AF0BA
:1026A000EFEC29F084C333F1FCEC29F073EC29F052
:1026B000200E0C6E00C10BF0EEEC07F000C12FF500
:1026C00005012F51000A06E005012F51010A02E021
:1026D000BDEC2CF004014C0E826F29EC0BF00401D0
:1026E0004D0E826F29EC0BF004012C0E826F29EC49
:1026F0000BF0AEEC29F02FC500F151EC29F033C1FD
:1027000082F40401300E822729EC0BF015EF1AF049
:10271000D2EF33F004014C0E826F29EC0BF0040170
:10272000630E826F29EC0BF067EC2BF004012C0E8A
:10273000826F29EC0BF09FEC13F015EF1AF0AEEC62
:1027400029F0B1C500F10101003B0F0E001751EC5B
:1027500029F033C182F40401300E822729EC0BF0FA
:10276000B1C500F101010F0E0101001751EC29F074
:1027700033C182F40401300E822729EC0BF00401EE
:102780002D0E826F29EC0BF0B0C500F10101003B6A
:102790000F0E001751EC29F033C182F40401300E02
:1027A000822729EC0BF0B0C500F101010F0E0101E9
:1027B000001751EC29F033C182F40401300E822756
:1027C00029EC0BF004012D0E826F29EC0BF0AFC544
:1027D00000F10101003B0F0E001751EC29F033C14D
:1027E00082F40401300E822729EC0BF0AFC500F112
:1027F00001010F0E0101001751EC29F033C182F4E1
:102800000401300E822729EC0BF00401200E826FA8
:1028100029EC0BF0AEC500F10F0E0101001751ECD1
:1028200029F033C182F40401300E822729EC0BF029
:102830000401200E826F29EC0BF0ADC500F10101FF
:102840000101003B0F0E001751EC29F033C182F457
:102850000401300E822729EC0BF0ADC500F1010117
:102860000F0E0101001751EC29F033C182F404016D
:10287000300E822729EC0BF004013A0E826F29EC0E
:102880000BF0ACC500F10101003B0F0E001751EC3D
:1028900029F033C182F40401300E822729EC0BF0B9
:1028A000ACC500F101010F0E0101001751EC29F038
:1028B00033C182F40401300E822729EC0BF00401AD
:1028C0003A0E826F29EC0BF0ABC500F10101003B21
:1028D0000F0E001751EC29F033C182F40401300EC1
:1028E000822729EC0BF0ABC500F101010F0E001798
:1028F00051EC29F033C182F40401300E822729EC17
:102900000BF0120084C3E8FF0F0BE83AE8CFB1F5F3
:1029100085C3E8FF0F0B0501B11387C3E8FF0F0B59
:10292000E83AE8CFB0F588C3E8FF0F0B0501B01314
:102930008AC3E8FF0F0BE83AE8CFAFF58BC3E8FF97
:102940000F0B0501AF138DC3E8FF0F0BE8CFAEF5FA
:102950008FC3E8FF0F0BE83AE8CFADF590C3E8FF6F
:102960000F0B0501AD1392C3E8FF0F0BE83AE8CF58
:10297000ACF593C3E8FF0F0B0501AC1395C3E8FF5B
:102980000F0BE83AE8CFABF596C3E8FF0F0B050154
:10299000AB13C6EC2BF004014C0E826F29EC0BF04C
:1029A0000401430E826F29EC0BF094EF13F00784BF
:1029B00093EC33F0AEEC29F02DC500F151EC29F089
:1029C00004014C0E826F29EC0BF00401300E826F73
:1029D00029EC0BF004012C0E826F29EC0BF031C1B5
:1029E00082F40401300E822729EC0BF032C182F40C
:1029F0000401300E822729EC0BF033C182F404016C
:102A0000300E822729EC0BF004012C0E826F29EC8A
:102A10000BF0AEEC29F02EC500F151EC29F031C1DC
:102A200082F40401300E822729EC0BF032C182F4CB
:102A30000401300E822729EC0BF033C182F404012B
:102A4000300E822729EC0BF0079415EF1AF00401E1
:102A50004C0E826F29EC0BF00401650E826F29EC9D
:102A60000BF0A6EC2DF015EF1AF004014C0E826F5E
:102A700029EC0BF00401450E826F29EC0BF0C3EC3E
:102A80002DF015EF1AF004014C0E826F29EC0BF0BB
:102A90000401620E826F29EC0BF0FDEC2DF015EFB6
:102AA0001AF004014C0E826F29EC0BF00401420E67
:102AB000826F29EC0BF0E0EC2DF015EF1AF0040119
:102AC0004C0E826F29EC0BF004015A0E826F29EC38
:102AD0000BF004012C0E826F29EC0BF093EC33F019
:102AE000AEEC29F005012E51130A06E005012E5126
:102AF000170A0DE090EF15F00101000E006F000EB7
:102B0000016F100E026F000E036F90EF15F00101C0
:102B1000000E006F000E016F000E026F010E036FBA
:102B20000101200E046F000E056F000E066F000EEF
:102B3000076FE4EC28F051EC29F02AC182F404017B
:102B4000300E822729EC0BF02BC182F40401300EE9
:102B5000822729EC0BF02CC182F40401300E82276D
:102B600029EC0BF02DC182F40401300E822729ECF0
:102B70000BF02EC182F40401300E822729EC0BF0F9
:102B80002FC182F40401300E822729EC0BF030C1F2
:102B900082F40401300E822729EC0BF031C182F45B
:102BA0000401300E822729EC0BF032C182F40401BB
:102BB000300E822729EC0BF033C182F40401300E71
:102BC000822729EC0BF015EF1AF0078404014C0E54
:102BD000826F29EC0BF00401310E826F29EC0BF0AF
:102BE00004012C0E826F29EC0BF025C500F126C5DF
:102BF00001F127C502F128C503F10101200E046F80
:102C0000000E056F000E066F000E076FE4EC28F053
:102C100051EC29F02AC182F40401300E822729ECFC
:102C20000BF02BC182F40401300E822729EC0BF04B
:102C30002CC182F40401300E822729EC0BF02DC147
:102C400082F40401300E822729EC0BF02EC182F4AD
:102C50000401300E822729EC0BF02FC182F404010D
:102C6000300E822729EC0BF030C182F40401300EC3
:102C7000822729EC0BF031C182F40401300E822747
:102C800029EC0BF032C182F40401300E822729ECCA
:102C90000BF033C182F40401300E822729EC0BF0D3
:102CA000079415EF1AF0078404014C0E826F29EC8B
:102CB0000BF00401320E826F29EC0BF0F3EC2FF0D5
:102CC000079415EF1AF0078404014C0E826F29EC6B
:102CD0000BF00401330E826F29EC0BF050EC30F056
:102CE0000794F0EF15F0078404014C0E826F29EC75
:102CF0000BF00401340E826F29EC0BF004012C0E52
:102D0000826F29EC0BF0EFEC29F084C32AF185C324
:102D10002BF186C32CF187C32DF188C32EF189C313
:102D20002FF18AC330F18BC331F18CC332F18DC3E3
:102D300033F10101296BFCEC29F073EC29F0200E32
:102D4000046F000E056F000E066F000E076FC4ECD7
:102D500028F000C121F501C122F502C123F503C10C
:102D600024F546EC33F034C5ABF535C5ACF536C5C6
:102D7000ADF537C5AEF538C5AFF539C5B0F53AC5CF
:102D8000B1F59FEC13F004012C0E826F29EC0BF0CF
:102D90003BC500F13CC501F13DC502F13EC503F163
:102DA0000101000E046F000E056F010E066F000E8C
:102DB000076FE4EC28F051EC29F02967E2EF16F0F8
:102DC000E7EF16F004012D0E826F29EC0BF030C1F5
:102DD00082F40401300E822729EC0BF031C182F419
:102DE0000401300E822729EC0BF004012E0E826FB5
:102DF00029EC0BF032C182F40401300E822729EC59
:102E00000BF033C182F40401300E822729EC0BF061
:102E100004012C0E826F29EC0BF0AEEC29F03FC5BB
:102E200000F140C501F12AEC23F004012C0E826F61
:102E300029EC0BF0AEEC29F041C500F151EC29F082
:102E400031C182F40401300E822729EC0BF032C12B
:102E500082F40401300E822729EC0BF033C182F496
:102E60000401300E822729EC0BF004012C0E826F36
:102E700029EC0BF00101036B026B48C501F147C55A
:102E800000F101AF49EF17F00101FF0E026FFF0ED5
:102E9000036F51EC29F0296750EF17F055EF17F049
:102EA00004012D0E826F29EC0BF02FC182F4040176
:102EB000300E822729EC0BF030C182F40401300E71
:102EC000822729EC0BF031C182F40401300E8227F5
:102ED00029EC0BF032C182F40401300E822729EC78
:102EE0000BF033C182F40401300E822729EC0BF081
:102EF00004012C0E826F29EC0BF00101036B026BB5
:102F00004AC501F149C500F101AF8CEF17F001018D
:102F1000FF0E026FFF0E036F51EC29F0296793EF4C
:102F200017F098EF17F004012D0E826F29EC0BF0CB
:102F30002FC182F40401300E822729EC0BF030C13E
:102F400082F40401300E822729EC0BF031C182F4A7
:102F50000401300E822729EC0BF032C182F4040107
:102F6000300E822729EC0BF033C182F40401300EBD
:102F7000822729EC0BF004012C0E826F29EC0BF058
:102F80000101036B026B4CC501F14BC500F101AFB0
:102F9000CFEF17F00101FF0E026FFF0E036F51EC30
:102FA00029F02967D6EF17F0DBEF17F004012D0E9B
:102FB000826F29EC0BF02FC182F40401300E8227BE
:102FC00029EC0BF030C182F40401300E822729EC89
:102FD0000BF031C182F40401300E822729EC0BF092
:102FE00032C182F40401300E822729EC0BF033C188
:102FF00082F40401300E822729EC0BF004012C0E20
:10300000826F29EC0BF00101036B026B4EC501F1DD
:103010004DC500F101AF12EF18F00101FF0E026F74
:10302000FF0E036F51EC29F0296719EF18F01EEF1E
:1030300018F004012D0E826F29EC0BF02FC182F4E1
:103040000401300E822729EC0BF030C182F4040118
:10305000300E822729EC0BF031C182F40401300ECE
:10306000822729EC0BF032C182F40401300E822752
:1030700029EC0BF033C182F40401300E822729ECD5
:103080000BF004012C0E826F29EC0BF00101036B95
:10309000026B50C501F14FC500F101AF55EF18F0BB
:1030A0000101FF0E026FFF0E036F51EC29F029673B
:1030B0005CEF18F061EF18F004012D0E826F29EC1F
:1030C0000BF02FC182F40401300E822729EC0BF0A3
:1030D00030C182F40401300E822729EC0BF031C19B
:1030E00082F40401300E822729EC0BF032C182F405
:1030F0000401300E822729EC0BF033C182F4040165
:10310000300E822729EC0BF004012C0E826F29EC83
:103110000BF00101036B026B52C501F151C500F1C7
:1031200001AF98EF18F00101FF0E026FFF0E036F61
:1031300051EC29F029679FEF18F0A4EF18F0040173
:103140002D0E826F29EC0BF02FC182F40401300E9A
:10315000822729EC0BF030C182F40401300E822763
:1031600029EC0BF031C182F40401300E822729ECE6
:103170000BF032C182F40401300E822729EC0BF0EF
:1031800033C182F40401300E822729EC0BF00401D4
:103190002C0E826F29EC0BF00101036B026B46C50C
:1031A00001F145C500F101AFDBEF18F00101FF0EA1
:1031B000026FFF0E036F51EC29F02967E2EF18F060
:1031C000E7EF18F004012D0E826F29EC0BF02FC1F0
:1031D00082F40401300E822729EC0BF030C182F416
:1031E0000401300E822729EC0BF031C182F4040176
:1031F000300E822729EC0BF032C182F40401300E2C
:10320000822729EC0BF033C182F40401300E8227AF
:1032100029EC0BF0079415EF1AF0EFEC29F085C3B9
:103220002AF186C32BF187C32CF188C32DF189C302
:103230002EF18AC32FF18BC330F18CC331F18DC3D2
:1032400032F18EC333F10101296BFCEC29F073ECF0
:1032500029F00101010E046F000E056F000E066FCC
:10326000000E076FB3EC28F0100E046F000E056F10
:10327000000E066F000E076FC4EC28F000C129F5A0
:1032800001C12AF502C12BF503C12CF57CEC2FF00E
:1032900004014C0E826F29EC0BF00401460E826F84
:1032A00029EC0BF004012C0E826F29EC0BF025C5E4
:1032B00000F126C501F127C502F128C503F101017E
:1032C000100E046F000E056F000E066F000E076FE4
:1032D000E4EC28F051EC29F02AC182F40401300E0C
:1032E000822729EC0BF02BC182F40401300E8227D7
:1032F00029EC0BF02CC182F40401300E822729EC5A
:103300000BF02DC182F40401300E822729EC0BF062
:103310002EC182F40401300E822729EC0BF02FC15C
:1033200082F40401300E822729EC0BF030C182F4C4
:103330000401300E822729EC0BF031C182F4040124
:10334000300E822729EC0BF032C182F40401300EDA
:10335000822729EC0BF033C182F40401300E82275E
:1033600029EC0BF015EF1AF00F9850EC30F000EF4D
:1033700022F004014C0E826F29EC0BF00401350E93
:10338000826F29EC0BF004012C0E826F29EC0BF0FC
:10339000AEEC29F00784B5C500F1079451EC29F093
:1033A00031C182F40401300E822729EC0BF032C1C6
:1033B00082F40401300E822729EC0BF033C182F431
:1033C0000401300E822729EC0BF015EF1AF013ECF4
:1033D00030F0AEEC29F033C500F151EC29F00401D6
:1033E0004C0E826F29EC0BF00401360E826F29EC33
:1033F0000BF004012C0E826F29EC0BF031C182F42A
:103400000401300E822729EC0BF032C182F4040152
:10341000300E822729EC0BF033C182F40401300E08
:10342000822729EC0BF015EF1AF033EC0BF000EFCC
:1034300022F004014C0E826F29EC0BF00401500EB7
:10344000826F29EC0BF004012C0E826F29EC0BF03B
:1034500085C32AF186C32BF187C32CF188C32DF1D4
:1034600089C32EF18AC32FF18BC330F18CC331F1A4
:103470008DC332F18EC333F10101FCEC29F073EC02
:1034800029F003018451530A0DE0030184514D0AD0
:1034900038E00401780E826F29EC0BF033EC0BF06E
:1034A00000EF22F00401530E826F29EC0BF0250E81
:1034B0000C6E00C10BF0EEEC07F0260E0C6E01C195
:1034C0000BF0EEEC07F0270E0C6E02C10BF0EEECE9
:1034D00007F0280E0C6E03C10BF0EEEC07F000C1F4
:1034E00053F501C154F502C155F503C156F500C1AC
:1034F00057F501C158F502C159F503C15AF5F6EF68
:103500001AF004014D0E826F29EC0BF0290E0C6E9F
:1035100000C10BF0EEEC07F000C15BF500C15CF5FB
:10352000F6EF1AF004014C0E826F29EC0BF0040147
:10353000540E826F29EC0BF004012C0E826F29ECE3
:103540000BF084C32AF185C32BF186C32CF187C30A
:103550002DF188C32EF189C32FF18AC330F18BC3BB
:1035600031F18DC332F18EC333F10101FCEC29F04E
:1035700073EC29F00101000E046F000E056F010EBF
:10358000066F000E076FC4EC28F0210E0C6E00C110
:103590000BF0EEEC07F0220E0C6E01C10BF0EEEC1E
:1035A00007F0230E0C6E02C10BF0EEEC07F0240EB8
:1035B0000C6E03C10BF0EEEC07F000C15DF501C12C
:1035C0005EF502C15FF503C160F5F6EF1AF0040184
:1035D0004C0E826F29EC0BF00401490E826F29EC2E
:1035E0000BF004012C0E826F29EC0BF0250E05EC7C
:1035F00008F0E8CF00F1260E05EC08F0E8CF01F165
:10360000270E05EC08F0E8CF02F1280E05EC08F0D3
:10361000E8CF03F151EC29F034EC27F00401730EEC
:10362000826F29EC0BF004012C0E826F29EC0BF059
:10363000AEEC29F0290E05EC08F0E8CF00F151ECD2
:1036400029F034EC27F00401730E826F29EC0BF0A3
:1036500004012C0E826F29EC0BF057C500F158C500
:1036600001F159C502F15AC503F151EC29F034ECCE
:1036700027F00401730E826F29EC0BF004012C0E6D
:10368000826F29EC0BF0AEEC29F05CC500F151EC37
:1036900029F034EC27F004016D0E826F29EC0BF059
:1036A00004012C0E826F29EC0BF05DC500F15EC5A4
:1036B00001F15FC502F160C503F11BEC22F00401CA
:1036C0002C0E826F29EC0BF033EC0BF000EF22F0A4
:1036D00083C32AF184C32BF185C32CF186C32DF15A
:1036E00087C32EF188C32FF189C330F18AC331F12A
:1036F0008BC332F18CC333F10101FCEC29F073EC84
:1037000029F0160E0C6E00C10BF0EEEC07F0170E50
:103710000C6E01C10BF0EEEC07F0180E0C6E02C13E
:103720000BF0EEEC07F0190E0C6E03C10BF0EEEC93
:1037300007F000C18AF101C18BF102C18CF103C114
:103740008DF100C18EF101C18FF102C190F103C171
:1037500091F14AEF1CF083C32AF184C32BF185C396
:103760002CF186C32DF187C32EF188C32FF189C3B5
:1037700030F18AC331F18BC332F18CC333F10101D3
:10378000FCEC29F073EC29F000C18AF101C18BF146
:1037900002C18CF103C18DF100C18EF101C18FF125
:1037A00002C190F103C191F14AEF1CF083C32AF1E9
:1037B00084C32BF185C32CF186C32DF187C32EF171
:1037C00088C32FF189C330F18AC331F18CC332F140
:1037D0008DC333F10101FCEC29F073EC29F00101F8
:1037E000000E046F000E056F010E066F000E076FCE
:1037F000C4EC28F01A0E0C6E00C10BF0EEEC07F0D2
:103800001B0E0C6E01C10BF0EEEC07F01C0E0C6EE3
:1038100002C10BF0EEEC07F01D0E0C6E03C10BF0B5
:10382000EEEC07F000C192F101C193F102C194F1F5
:1038300003C195F14AEF1CF083C32AF184C32BF135
:1038400085C32CF186C32DF187C32EF188C32FF1D8
:1038500089C330F18AC331F18CC332F18DC333F1A6
:103860000101FCEC29F073EC29F00101000E046F5A
:10387000000E056F010E066F000E076FC4EC28F0F6
:1038800000C192F101C193F102C194F103C195F11C
:103890004AEF1CF0160E05EC08F0E8CF00F1170E09
:1038A00005EC08F0E8CF01F1180E05EC08F0E8CFC0
:1038B00002F1190E05EC08F0E8CF03F151EC29F004
:1038C00034EC27F00401730E826F29EC0BF0040135
:1038D0002C0E826F29EC0BF08AC100F18BC101F133
:1038E0008CC102F18DC103F151EC29F034EC27F0C9
:1038F0000401730E826F29EC0BF004012C0E826F11
:1039000029EC0BF01A0E05EC08F0E8CF00F11B0EC5
:1039100005EC08F0E8CF01F11C0E05EC08F0E8CF4B
:1039200002F11D0E05EC08F0E8CF03F11BEC22F0CC
:1039300004012C0E826F29EC0BF092C100F193C1AF
:1039400001F194C102F195C103F11BEC22F033ECBB
:103950000BF000EF22F00401690E826F29EC0BF0EE
:1039600004012C0E826F29EC0BF00101040E006F94
:10397000000E016F000E026F000E036F51EC29F074
:103980002CC182F40401300E822729EC0BF02DC1EA
:1039900082F40401300E822729EC0BF02EC182F450
:1039A0000401300E822729EC0BF02FC182F40401B0
:1039B000300E822729EC0BF030C182F40401300E66
:1039C000822729EC0BF031C182F40401300E8227EA
:1039D00029EC0BF032C182F40401300E822729EC6D
:1039E0000BF033C182F40401300E822729EC0BF076
:1039F00004012C0E826F29EC0BF001010B0E006FFD
:103A0000000E016F000E026F000E036F51EC29F0E3
:103A10002CC182F40401300E822729EC0BF02DC159
:103A200082F40401300E822729EC0BF02EC182F4BF
:103A30000401300E822729EC0BF02FC182F404011F
:103A4000300E822729EC0BF030C182F40401300ED5
:103A5000822729EC0BF031C182F40401300E822759
:103A600029EC0BF032C182F40401300E822729ECDC
:103A70000BF033C182F40401300E822729EC0BF0E5
:103A800004012C0E826F29EC0BF001011F0E006F58
:103A9000000E016F000E026F000E036F51EC29F053
:103AA0002CC182F40401300E822729EC0BF02DC1C9
:103AB00082F40401300E822729EC0BF02EC182F42F
:103AC0000401300E822729EC0BF02FC182F404018F
:103AD000300E822729EC0BF030C182F40401300E45
:103AE000822729EC0BF031C182F40401300E8227C9
:103AF00029EC0BF032C182F40401300E822729EC4C
:103B00000BF033C182F40401300E822729EC0BF054
:103B100004012C0E826F29EC0BF0200EF86EF76A70
:103B2000F66A04010900F5CF82F429EC0BF00900D4
:103B3000F5CF82F429EC0BF00900F5CF82F429ECE3
:103B40000BF00900F5CF82F429EC0BF00900F5CF5A
:103B500082F429EC0BF00900F5CF82F429EC0BF08C
:103B60000900F5CF82F429EC0BF00900F5CF82F4BF
:103B700029EC0BF033EC0BF000EF22F08351630AD9
:103B8000D8A400EF22F08451610AD8A400EF22F0FB
:103B900085516C0AD8A400EF22F08651410A42E018
:103BA0008651440A1BE08651420AD8B425EF1EF024
:103BB0008651350AD8B48AEF23F08651360AD8B434
:103BC000DFEF23F08651370AD8B448EF24F086514E
:103BD000380AD8B4A6EF24F000EF22F00798079A2D
:103BE00004017A0E826F29EC0BF00401780E826FCB
:103BF00029EC0BF00401640E826F29EC0BF081A814
:103C000009EF1EF00401550E826F29EC0BF00EEF48
:103C10001EF004014C0E826F29EC0BF033EC0BF01C
:103C200000EF22F00788079A04017A0E826F29ECD0
:103C30000BF00401410E826F29EC0BF00401610EC0
:103C4000826F29EC0BF0FFEF1DF00798078A040143
:103C50007A0E826F29EC0BF00401420E826F29EC80
:103C60000BF00401610E826F29EC0BF0FFEF1DF0E9
:103C70000101666743EF1EF0676743EF1EF0686758
:103C800043EF1EF069675BEF1EF04F674FEF1EF0CA
:103C900050674FEF1EF051674FEF1EF052675BEF1A
:103CA0001EF00101000E006F000E016F000E026F8A
:103CB000000E036F12000101620E046F010E056F0A
:103CC000000E066F000E076F66C100F167C101F1BB
:103CD00068C102F169C103F1B3EC28F003BFDFEF63
:103CE0001EF00101000E046FA80E056F550E066F41
:103CF000020E076F66C100F167C101F168C102F1F0
:103D000069C103F166C186F167C187F168C188F1B5
:103D100069C189F1B3EC28F003BF98EF1EF00101EF
:103D2000000E866FA80E876F550E886F020E896F82
:103D30000E0E05EC08F0E8CF18F10F0E05EC08F0B8
:103D4000E8CF19F1100E05EC08F0E8CF1AF1110ECA
:103D500005EC08F0E8CF1BF1FCEC27F086C104F17C
:103D600087C105F188C106F189C107F1B3EC28F0DC
:103D70000782C0EC27F0FCEC27F00792C0EC27F09C
:103D800086C100F187C101F188C102F189C103F147
:103D90000792C0EC27F0CC0E046FE00E056F870E83
:103DA000066F050E076FB3EC28F000C118F101C1D2
:103DB00019F102C11AF103C11BF117EF1FF0010144
:103DC000800E006F1A0E016F060E026F000E036F59
:103DD0004FC104F150C105F151C106F152C107F1C3
:103DE000B3EC28F003AFF8EF1EF0AEEC29F01200B0
:103DF0000E0E05EC08F0E8CF18F10F0E05EC08F0F8
:103E0000E8CF19F1100E05EC08F0E8CF1AF1110E09
:103E100005EC08F0E8CF1BF14FC100F150C101F1F2
:103E200051C102F152C103F10782C0EC27F018C161
:103E300000F119C101F11AC102F11BC103F1120015
:103E40000401730E826F29EC0BF004012C0E826FBB
:103E500029EC0BF0078462C166F163C167F164C1AC
:103E600068F165C169F14BC14FF14CC150F14DC1D1
:103E700051F14EC152F157C159F158C15AF107944D
:103E800046EC1FF033EC0BF000EF22F066C100F1BE
:103E900067C101F168C102F169C103F1010151EC8F
:103EA00029F034EC27F00401630E826F29EC0BF04B
:103EB00004012C0E826F29EC0BF04FC100F150C1B0
:103EC00001F151C102F152C103F1010151EC29F09C
:103ED00034EC27F00401660E826F29EC0BF004012C
:103EE0002C0E826F29EC0BF0AEEC29F059C100F1D9
:103EF0005AC101F1010151EC29F034EC27F0040121
:103F0000740E826F29EC0BF0120010820401530E24
:103F1000826F29EC0BF004012C0E826F29EC0BF060
:103F200083C32AF184C32BF185C32CF186C32DF101
:103F300087C32EF188C32FF189C330F18AC331F1D1
:103F40008BC332F18CC333F10101FCEC29F073EC2B
:103F500029F000C166F101C167F102C168F103C136
:103F600069F18EC32AF18FC32BF190C32CF191C359
:103F70002DF192C32EF193C32FF194C330F195C369
:103F800031F196C332F197C333F10101FCEC29F012
:103F900073EC29F000C14FF101C150F102C151F1A0
:103FA00003C152F1EFEC29F099C32FF19AC330F11C
:103FB0009BC331F19CC332F19DC333F10101FCEC91
:103FC00029F073EC29F000C159F101C15AF146EC16
:103FD0001FF004012C0E826F29EC0BF0F7EF1FF09D
:103FE0008251520A03E10F82F7EF1FF00F928251C4
:103FF000750A03E11084FEEF1FF010948251550AF8
:1040000003E1108605EF20F01096078410B262EFEE
:1040100020F010A44EEF20F0B6C166F1B7C167F1F1
:10402000B8C168F1B9C169F1BAC16AF1BBC16BF13C
:10403000BCC16CF1BDC16DF1BEC16EF1BFC16FF10C
:10404000C0C170F1C1C171F1C2C172F1C3C173F1DC
:10405000C4C174F1C5C175F1C6C176F1C7C177F1AC
:10406000C8C178F1C9C179F1CAC17AF1CBC17BF17C
:10407000CCC17CF1CDC17DF1CEC17EF1CFC17FF14C
:10408000D0C180F1D1C181F1D2C182F1D3C183F11C
:10409000D4C184F1D5C185F156EF20F062C166F13B
:1040A00063C167F164C168F165C169F14BC14FF14A
:1040B0004CC150F14DC151F14EC152F157C159F1AE
:1040C00058C15AF107940FA084EF20F001019267C4
:1040D00071EF20F0936771EF20F0946771EF20F09B
:1040E000956775EF20F084EF20F038EC1EF092C158
:1040F00004F193C105F194C106F195C107F1B3EC48
:1041000028F003BFC8EF21F038EC1EF00101000ECB
:10411000046F000E056F010E066F000E076FE4ECD2
:1041200028F010A49BEF20F00401750E826F29EC9B
:104130000BF0A0EF20F00401720E826F29EC0BF05F
:1041400004012C0E826F29EC0BF051EC29F0296749
:10415000AFEF20F00401200E826FB2EF20F00401D7
:104160002D0E826F29EC0BF030C182F40401300E69
:10417000822729EC0BF031C182F40401300E822732
:1041800029EC0BF004012E0E826F29EC0BF032C1EA
:1041900082F40401300E822729EC0BF033C182F443
:1041A0000401300E822729EC0BF004016D0E826FA2
:1041B00029EC0BF004012C0E826F29EC0BF04FC19F
:1041C00000F150C101F151C102F152C103F10101ED
:1041D00051EC29F034EC27F00401480E826F29ECF1
:1041E0000BF004017A0E826F29EC0BF004012C0E07
:1041F000826F29EC0BF066C100F167C101F168C163
:1042000002F169C103F1010151EC29F034EC27F00E
:104210000401630E826F29EC0BF004012C0E826FF7
:1042200029EC0BF066C100F167C101F168C102F130
:1042300069C103F101010A0E046F000E056F000E43
:10424000066F000E076FC4EC28F0000E046F120E0C
:10425000056F000E066F000E076FE4EC28F051ECBE
:1042600029F02AC182F40401300E822729EC0BF0D8
:104270002BC182F40401300E822729EC0BF02CC1F3
:1042800082F40401300E822729EC0BF02DC182F458
:104290000401300E822729EC0BF02EC182F40401B8
:1042A000300E822729EC0BF02FC182F40401300E6E
:1042B000822729EC0BF030C182F40401300E8227F2
:1042C00029EC0BF004012E0E826F29EC0BF031C1AA
:1042D00082F40401300E822729EC0BF032C182F403
:1042E0000401300E822729EC0BF033C182F4040163
:1042F000300E822729EC0BF00401730E826F29EC3B
:104300000BF004012C0E826F29EC0BF0AEEC29F0BF
:1043100059C100F15AC101F12AEC23F00FB294EF18
:1043200021F00FA0C6EF21F004012C0E826F29ECC2
:104330000BF0200EF86EF76AF66A04010900F5CF5B
:1043400082F429EC0BF00900F5CF82F429EC0BF094
:104350000900F5CF82F429EC0BF00900F5CF82F4C7
:1043600029EC0BF00900F5CF82F429EC0BF00900E1
:10437000F5CF82F429EC0BF00900F5CF82F429EC9B
:104380000BF00900F5CF82F429EC0BF033EC0BF0C5
:104390000F9000EF22F00401630E826F29EC0BF006
:1043A00004012C0E826F29EC0BF006EC22F00401C4
:1043B0002C0E826F29EC0BF079EC22F004012C0E0C
:1043C000826F29EC0BF0F5EC22F004012C0E826FC9
:1043D00029EC0BF00101F80E006FCD0E016F660E97
:1043E000026F030E036F1BEC22F004012C0E826F90
:1043F00029EC0BF00BEC23F033EC0BF000EF22F088
:104400000301C26B079010920FEF25F0D8900E0EAB
:1044100005EC08F0E8CF00F10F0E05EC08F0E8CF4E
:1044200001F1100E05EC08F0E8CF02F1110E05ECD9
:1044300008F0E8CF03F10101000E046F000E056FD4
:10444000010E066F000E076FE4EC28F051EC29F026
:104450002AC182F40401300E822729EC0BF02BC113
:1044600082F40401300E822729EC0BF02CC182F477
:104470000401300E822729EC0BF02DC182F40401D7
:10448000300E822729EC0BF02EC182F40401300E8D
:10449000822729EC0BF02FC182F40401300E822711
:1044A00029EC0BF030C182F40401300E822729EC94
:1044B0000BF031C182F40401300E822729EC0BF09D
:1044C00004012E0E826F29EC0BF032C182F404013C
:1044D000300E822729EC0BF033C182F40401300E38
:1044E000822729EC0BF004016D0E826F29EC0BF092
:1044F0001200120E05EC08F0E8CF00F1130E05ECE7
:1045000008F0E8CF01F1140E05EC08F0E8CF02F155
:10451000150E05EC08F0E8CF03F101010A0E046F57
:10452000000E056F000E066F000E076FC4EC28F03A
:10453000000E046F120E056F000E066F000E076F5F
:10454000E4EC28F051EC29F02AC182F40401300E89
:10455000822729EC0BF02BC182F40401300E822754
:1045600029EC0BF02CC182F40401300E822729ECD7
:104570000BF02DC182F40401300E822729EC0BF0E0
:104580002EC182F40401300E822729EC0BF02FC1DA
:1045900082F40401300E822729EC0BF030C182F442
:1045A0000401300E822729EC0BF004012E0E826FDD
:1045B00029EC0BF031C182F40401300E822729EC82
:1045C0000BF032C182F40401300E822729EC0BF08B
:1045D00033C182F40401300E822729EC0BF0040170
:1045E000730E826F29EC0BF012000A0E05EC08F036
:1045F000E8CF00F10B0E05EC08F0E8CF01F10C0E4E
:1046000005EC08F0E8CF02F10D0E05EC08F0E8CF5C
:1046100003F12AEF23F0060E05EC08F0E8CF00F1D5
:10462000070E05EC08F0E8CF01F1080E05EC08F0E4
:10463000E8CF02F1090E05EC08F0E8CF03F12AEF0C
:1046400023F00101AEEC29F0078457C100F158C1F5
:1046500001F107940101E80E046F800E056F000E52
:10466000066F000E076FC4EC28F0000E046F040EF6
:10467000056F000E066F000E076FE4EC28F0880E41
:10468000046F130E056F000E066F000E076FB3EC7C
:1046900028F00A0E046F000E056F000E066F000E64
:1046A000076FE4EC28F051EC29F0010129675EEF77
:1046B00023F00401200E826F61EF23F004012D0E20
:1046C000826F29EC0BF030C182F40401300E822796
:1046D00029EC0BF031C182F40401300E822729EC61
:1046E0000BF032C182F40401300E822729EC0BF06A
:1046F00004012E0E826F29EC0BF033C182F4040109
:10470000300E822729EC0BF00401430E826F29EC56
:104710000BF0120087C32AF188C32BF189C32CF157
:104720008AC32DF18BC32EF18CC32FF18DC330F1D1
:104730008EC331F190C332F191C333F10101296B82
:10474000FCEC29F073EC29F00101000E046F000E5F
:10475000056F010E066F000E076FC4EC28F00E0EF9
:104760000C6E00C10BF0EEEC07F00F0E0C6E01C1E9
:104770000BF0EEEC07F0100E0C6E02C10BF0EEEC3D
:1047800007F0110E0C6E03C10BF0EEEC07F0040104
:104790007A0E826F29EC0BF004012C0E826F29EC4B
:1047A0000BF00401350E826F29EC0BF004012C0E86
:1047B000826F29EC0BF006EC22F00EEF1EF087C39F
:1047C0002AF188C32BF189C32CF18AC32DF18BC345
:1047D0002EF18CC32FF18DC330F18EC331F190C314
:1047E00032F191C333F10101296BFCEC29F073EC38
:1047F00029F0880E046F130E056F000E066F000E71
:10480000076FB8EC28F0000E046F040E056F000E61
:10481000066F000E076FC4EC28F00101E80E046F6C
:10482000800E056F000E066F000E076FE4EC28F097
:104830000A0E0C6E00C10BF0EEEC07F00B0E0C6EC6
:1048400001C10BF0EEEC07F00C0E0C6E02C10BF088
:10485000EEEC07F00D0E0C6E03C10BF0EEEC07F062
:1048600004017A0E826F29EC0BF004012C0E826F8A
:1048700029EC0BF00401360E826F29EC0BF00401D9
:104880002C0E826F29EC0BF0F5EC22F00EEF1EF0EF
:1048900087C32AF188C32BF189C32CF18AC32DF178
:1048A0008BC32EF18CC32FF18DC330F18FC331F147
:1048B00090C332F191C333F10101FCEC29F073ECA8
:1048C00029F0000E046F120E056F000E066F000E29
:1048D000076FC4EC28F001010A0E046F000E056F8B
:1048E000000E066F000E076FE4EC28F0120E0C6E3F
:1048F00000C10BF0EEEC07F0130E0C6E01C10BF0D3
:10490000EEEC07F0140E0C6E02C10BF0EEEC07F0AB
:10491000150E0C6E03C10BF0EEEC07F004017A0EDD
:10492000826F29EC0BF004012C0E826F29EC0BF046
:104930000401370E826F29EC0BF004012C0E826FFC
:1049400029EC0BF079EC22F00EEF1EF087C32AF170
:1049500088C32BF189C32CF18AC32DF18BC32EF1AF
:104960008CC32FF18DC330F18EC331F190C332F17E
:1049700091C333F10101296BFCEC29F073EC29F0B0
:10498000880E046F130E056F000E066F000E076F82
:10499000B8EC28F0000E046F040E056F000E066FD1
:1049A000000E076FC4EC28F00101E80E046F800EC2
:1049B000056F000E066F000E076FE4EC28F0060E80
:1049C0000C6E00C10BF0EEEC07F0070E0C6E01C18F
:1049D0000BF0EEEC07F0080E0C6E02C10BF0EEECE3
:1049E00007F0090E0C6E03C10BF0EEEC07F00401AA
:1049F0007A0E826F29EC0BF004012C0E826F29ECE9
:104A00000BF00401380E826F29EC0BF004012C0E20
:104A1000826F29EC0BF00BEC23F00EEF1EF081A857
:104A2000CDEF25F007A886EF25F00101800E006F7D
:104A30001A0E016F060E026F000E036F4BC104F1D8
:104A40004CC105F14DC106F14EC107F1B3EC28F0A0
:104A500003BFCDEF25F02EEC27F04BC100F14CC188
:104A600001F14DC102F14EC103F10782C0EC27F004
:104A700018C104F119C105F11AC106F11BC107F1F2
:104A8000F80E006FCD0E016F660E026F030E036FFE
:104A9000B3EC28F00E0E0C6E00C10BF0EEEC07F03C
:104AA0000F0E0C6E01C10BF0EEEC07F0100E0C6E49
:104AB00002C10BF0EEEC07F0110E0C6E03C10BF00F
:104AC000EEEC07F007840101AEEC29F057C100F1CC
:104AD00058C101F107940A0E0C6E00C10BF0EEEC08
:104AE00007F00B0E0C6E01C10BF0EEEC07F00C0E94
:104AF0000C6E02C10BF0EEEC07F00D0E0C6E03C154
:104B00000BF0EEEC07F00798CDEF25F007AACDEFFC
:104B100025F007840101AEEC29F057C100F158C11E
:104B200001F10794060E0C6E00C10BF0EEEC07F0DD
:104B3000070E0C6E01C10BF0EEEC07F0080E0C6EC8
:104B400002C10BF0EEEC07F0090E0C6E03C10BF086
:104B5000EEEC07F0078462C100F163C101F164C1AA
:104B600002F165C103F10794120E0C6E00C10BF047
:104B7000EEEC07F0130E0C6E01C10BF0EEEC07F03B
:104B8000140E0C6E02C10BF0EEEC07F0150E0C6E5D
:104B900003C10BF0EEEC07F0079A04018051811974
:104BA0007F0B0BE09EA809D014EE00F081517F0B23
:104BB000E126E750812B0F01AD6E05012F51010A4F
:104BC00013E081AAF4EF25F005012F51000A0AE055
:104BD0000FB8F4EF25F005013067F4EF25F00FB8BA
:104BE000F4EF25F0D2EF33F081B809EF26F017EC9F
:104BF0002CF005012F51020A02E009EF26F05C2F8C
:104C000009EF26F05BC55CF50501010E306F3C0E27
:104C1000316F92EF0AF006013251385D3351D8A05E
:104C2000010F395D800BD8A41AEF26F032C638F692
:104C300033C639F6120006013251365D3351D8A021
:104C4000010F375D800BD8B42AEF26F032C636F656
:104C500033C637F6120007841AC632F61BC633F67F
:104C60001CC638F61DC639F60BEC26F01EC632F609
:104C70001FC633F60BEC26F020C632F621C633F6FB
:104C80000BEC26F01AC632F61BC633F61CC636F6F7
:104C90001DC637F61BEC26F01EC632F61FC633F6CD
:104CA0001BEC26F020C632F621C633F61BEC26F0AC
:104CB0003851365F3951D8A03929375FAEEC29F029
:104CC00036C600F137C601F1BAEC29F000C13AF658
:104CD00001C13BF622C632F623C633F624C638F6A7
:104CE00025C639F60BEC26F026C632F627C633F673
:104CF0000BEC26F028C632F629C633F60BEC26F06C
:104D000022C632F623C633F624C636F625C637F653
:104D10001BEC26F026C632F627C633F61BEC26F02F
:104D200028C632F629C633F61BEC26F03851365F1A
:104D30003951D8A03929375FAEEC29F036C600F1D9
:104D400037C601F1BAEC29F000C13CF601C13DF6CD
:104D50002AC632F62BC633F62CC638F62DC639F6DF
:104D60000BEC26F02EC632F62FC633F60BEC26F0EF
:104D700030C632F631C633F60BEC26F02AC632F6D0
:104D80002BC633F62CC636F62DC637F61BEC26F0AE
:104D90002EC632F62FC633F61BEC26F030C632F69E
:104DA00031C633F61BEC26F03851365F3951D8A0A6
:104DB0003929375FAEEC29F036C600F137C601F16C
:104DC000BAEC29F000C13EF601C13FF63AC632F610
:104DD0003BC633F63CC636F63DC637F61BEC26F02E
:104DE0003EC632F63FC633F61BEC26F0079412009F
:104DF00018C100F119C101F11AC102F11BC103F17F
:104E0000000E046F000E056F010E066F000E076F97
:104E1000E4EC28F029A123EF27F02051D8B423EFA8
:104E200027F018C100F119C101F11AC102F11BC12B
:104E300003F1000E046F000E056F0A0E066F000EE0
:104E4000076FE4EC28F01200010104510013055132
:104E50000113065102130751031312000101186BCD
:104E6000196B1A6B1B6B12002AC182F40401300EFD
:104E7000822729EC0BF02BC182F40401300E82272B
:104E800029EC0BF02CC182F40401300E822729ECAE
:104E90000BF02DC182F40401300E822729EC0BF0B7
:104EA0002EC182F40401300E822729EC0BF02FC1B1
:104EB00082F40401300E822729EC0BF030C182F419
:104EC0000401300E822729EC0BF031C182F4040179
:104ED000300E822729EC0BF032C182F40401300E2F
:104EE000822729EC0BF033C182F40401300E8227B3
:104EF00029EC0BF012002FC182F40401300E82273E
:104F000029EC0BF030C182F40401300E822729EC29
:104F10000BF031C182F40401300E822729EC0BF032
:104F200032C182F40401300E822729EC0BF033C128
:104F300082F40401300E822729EC0BF01200060ED9
:104F4000116E060E126E060E136E112EA5EF27F0CF
:104F5000122EA5EF27F0132EA5EF27F08B84020E5B
:104F6000116E020E126E020E136E112EB5EF27F0A7
:104F7000122EB5EF27F0132EB5EF27F08B94120009
:104F80000101005305E1015303E1025301E1002B4C
:104F900083EC28F0AEEC29F03951006F3A51016FE3
:104FA000420E046F4B0E056F000E066F000E076F6A
:104FB000C4EC28F000C104F101C105F102C106F101
:104FC00003C107F118C100F119C101F11AC102F1C1
:104FD0001BC103F107B2F1EF27F0B8EC28F0F3EFB3
:104FE00027F0B3EC28F000C118F101C119F102C19A
:104FF0001AF103C11BF11200AEEC29F059C100F106
:105000005AC101F1060E05EC08F0E8CF04F1070ED5
:1050100005EC08F0E8CF05F1080E05EC08F0E8CF44
:1050200006F1090E05EC08F0E8CF07F1B3EC28F023
:1050300000C124F101C125F102C126F103C127F10C
:10504000290E046F000E056F000E066F000E076F2D
:10505000C4EC28F0EE0E046F430E056F000E066FD1
:10506000000E076FB8EC28F024C104F125C105F14A
:1050700026C106F127C107F1C4EC28F000C11CF1DC
:1050800001C11DF102C11EF103C11FF1120E05EC99
:1050900008F0E8CF04F1130E05EC08F0E8CF05F1B5
:1050A000140E05EC08F0E8CF06F1150E05EC08F03B
:1050B000E8CF07F10D0E006F000E016F000E026FBA
:1050C000000E036FC4EC28F0180E046F000E056F7D
:1050D000000E066F000E076FE4EC28F01CC104F10F
:1050E0001DC105F11EC106F11FC107F1B8EC28F082
:1050F0006A0E046F2A0E056F000E066F000E076F12
:10510000B3EC28F01200BF0EFA6E200E3A6F396B26
:10511000D8900037013702370337D8B094EF28F022
:105120003A2F89EF28F039073A070353D8B4120011
:105130000331070B80093F6F03390F0B010F396FE4
:1051400080EC5FF0406F390580EC5FF0405D405FC0
:10515000396B3F33D8B0392739333FA9A9EF28F04D
:105160004051392712000101D3EC29F0D8B01200C8
:10517000010103510719346F96EC29F0D8900751BB
:10518000031934AF800F12000101346BBAEC29F01F
:10519000D8A0D0EC29F0D8B01200A5EC29F0AEECE4
:1051A00029F01F0E366FE6EC29F00B35D8B096ECDF
:1051B00029F0D8A00335D8B01200362FD3EF28F04D
:1051C00034B1BDEC29F012000101346B045105111A
:1051D000061107110008D8A0BAEC29F0D8A0D0EC2D
:1051E00029F0D8B01200086B096B0A6B0B6BE6EC68
:1051F00029F01F0E366FE6EC29F007510B5DD8A49D
:105200000EEF29F006510A5DD8A40EEF29F00551E2
:10521000095DD8A40EEF29F00451085DD8A021EF54
:1052200029F00451085F0551D8A0053D095F0651DA
:10523000D8A0063D0A5F0751D8A0073D0B5FD89064
:105240000081362FFBEF28F034B1BDEC29F0346B30
:10525000BAEC29F0D890EAEC29F007510B5DD8A4FC
:105260003EEF29F006510A5DD8A43EEF29F0055122
:10527000095DD8A43EEF29F00451085DD8A04DEF98
:1052800029F0003F4DEF29F0013F4DEF29F0023F9B
:105290004DEF29F0032BD8B4120034B1BDEC29F046
:1052A00012000101346BBAEC29F0D8B01200EFEC17
:1052B00029F0200E366F003701370237033711EE21
:1052C00033F00A0E376FE7360A0EE75CD8B0E76EA8
:1052D000E552372F63EF29F0362F5BEF29F034B119
:1052E0002981D890120001010A0E346F200E366F0A
:1052F00011EE29F03451376F0A0ED890E652D8B02B
:10530000E726E732372F7EEF29F0033302330133EC
:105310000033362F78EF29F0E750FF0FD8A0033580
:10532000D8B0120029B1BDEC29F0120004510027B9
:105330000551D8B0053D01270651D8B0063D0227DA
:105340000751D8B0073D032712000051086F0151E3
:10535000096F02510A6F03510B6F12000101006BBC
:10536000016B026B036B12000101046B056B066B92
:10537000076B12000335D8A012000351800B001FE9
:10538000011F021F031F003FCDEF29F0013FCDEFAA
:1053900029F0023FCDEF29F0032B342B0325120017
:1053A0000735D8A012000751800B041F051F061FE8
:1053B000071F043FE3EF29F0053FE3EF29F0063F25
:1053C000E3EF29F0072B342B0725120000370137B4
:1053D00002370337083709370A370B371200010144
:1053E000296B2A6B2B6B2C6B2D6B2E6B2F6B306B01
:1053F000316B326B336B120001012A510F0B2A6F94
:105400002B510F0B2B6F2C510F0B2C6F2D510F0BA2
:105410002D6F2E510F0B2E6F2F510F0B2F6F305101
:105420000F0B306F31510F0B316F32510F0B326F49
:1054300033510F0B336F1200899C000EC76E200E84
:10544000C66E9E96C69EC50EC96EFF0E9EB602D053
:10545000E82EFCD79E96C69E000EC96EFF0E9EB625
:1054600002D0E82EFCD7C9CF00F69E96C69E000E4D
:10547000C96EFF0E9EB602D0E82EFCD7C9CF01F64A
:10548000898C1200000EC76E200EC66E899C9E96F7
:10549000C69EC80EC96EFF0E9EB602D0E82EFCD77F
:1054A0009E96C69E000EC96EFF0E9EB602D0E82ED6
:1054B000FCD7C9CF02F69E96C69E000EC96EFF0E9F
:1054C0009EB602D0E82EFCD7C9CF03F6898C899C02
:1054D0009E96C69ECA0EC96EFF0E9EB602D0E82EDC
:1054E000FCD79E96C69E000EC96EFF0E9EB602D0D9
:1054F000E82EFCD7C9CF0AF69E96C69E000EC96E4E
:10550000FF0E9EB602D0E82EFCD7C9CF0BF6898CD1
:10551000899C9E96C69ECC0EC96EFF0E9EB602D08A
:10552000E82EFCD79E96C69E000EC96EFF0E9EB654
:1055300002D0E82EFCD7C9CF12F69E96C69E000E6A
:10554000C96EFF0E9EB602D0E82EFCD7C9CF13F667
:10555000898C1200000EC76E200EC66E899C9E9626
:10556000C69EE80EC96EFF0E9EB602D0E82EFCD78E
:105570009E96C69E000EC96EFF0E9EB602D0E82E05
:10558000FCD7C9CF1AF69E96C69E000EC96EFF0EB6
:105590009EB602D0E82EFCD7C9CF1BF6898C899C19
:1055A0009E96C69EEA0EC96EFF0E9EB602D0E82EEB
:1055B000FCD79E96C69E000EC96EFF0E9EB602D008
:1055C000E82EFCD7C9CF22F69E96C69E000EC96E65
:1055D000FF0E9EB602D0E82EFCD7C9CF23F6898CE9
:1055E000899C9E96C69EEC0EC96EFF0E9EB602D09A
:1055F000E82EFCD79E96C69E000EC96EFF0E9EB684
:1056000002D0E82EFCD7C9CF2AF69E96C69E000E81
:10561000C96EFF0E9EB602D0E82EFCD7C9CF2BF67E
:10562000898C1200000EC76E200EC66E899C9E9655
:10563000C69E240EC96EFF0E9EB602D0E82EFCD781
:105640009E96C69EE40EC96EFF0E9EB602D0E82E50
:10565000FCD7898C899C9E96C69E200EC96EFF0E33
:105660009EB602D0E82EFCD79E96C69E5F0EC96EEF
:10567000FF0E9EB602D0E82EFCD7898C899C9E96A0
:10568000C69E210EC96EFF0E9EB602D0E82EFCD734
:105690009E96C69EC00EC96EFF0E9EB602D0E82E24
:1056A000FCD7898C899C9E96C69E260EC96EFF0EDD
:1056B0009EB602D0E82EFCD79E96C69E000EC96EFE
:1056C000FF0E9EB602D0E82EFCD7898C120089848A
:1056D000000EC76E220EC66E9E96C69E000EC96E46
:1056E000FF0E9EB602D0E82EFCD79E96C69E000EF8
:1056F000C96EFF0E9EB602D0E82EFCD7C9CFABF51F
:105700009E96C69E000EC96EFF0E9EB602D0E82E73
:10571000FCD7C9CFACF59E96C69E000EC96EFF0E93
:105720009EB602D0E82EFCD7C9CFADF59E96C69E98
:10573000000EC96EFF0E9EB602D0E82EFCD7C9CF70
:10574000AEF59E96C69E000EC96EFF0E9EB602D0A6
:10575000E82EFCD7C9CFAFF59E96C69E000EC96E47
:10576000FF0E9EB602D0E82EFCD7C9CFB0F59E96AC
:10577000C69E000EC96EFF0E9EB602D0E82EFCD764
:10578000C9CFB1F589941AEC2EF012008984000E6D
:10579000C76E220EC66E9E96C69E800EC96EFF0E06
:1057A0009EB602D0E82EFCD79E96C69EABC5C9FF1A
:1057B000FF0E9EB602D0E82EFCD79E96C69EACC5C4
:1057C000C9FFFF0E9EB602D0E82EFCD79E96C69E5D
:1057D000ADC5C9FFFF0E9EB602D0E82EFCD79E963F
:1057E000C69EAEC5C9FFFF0E9EB602D0E82EFCD7FE
:1057F0009E96C69EAFC5C9FFFF0E9EB602D0E82E8C
:10580000FCD79E96C69EB0C5C9FFFF0E9EB602D0BD
:10581000E82EFCD79E96C69EB1C5C9FFFF0E9EB668
:1058200002D0E82EFCD789941AEC2EF0120089845D
:10583000000EC76E220EC66E9E96C69E070EC96EDD
:10584000FF0E9EB602D0E82EFCD79E96C69E000E96
:10585000C96EFF0E9EB602D0E82EFCD7C9CFABF5BD
:105860009E96C69E000EC96EFF0E9EB602D0E82E12
:10587000FCD7C9CFACF59E96C69E000EC96EFF0E32
:105880009EB602D0E82EFCD7C9CFADF59E96C69E37
:10589000000EC96EFF0E9EB602D0E82EFCD7C9CF0F
:1058A000AEF589941AEC2EF08984000EC76E220E94
:1058B000C66E9E96C69E0F0EC96EFF0E9EB602D095
:1058C000E82EFCD79E96C69E000EC96EFF0E9EB6B1
:1058D00002D0E82EFCD7C9CFB3F589941AEC2EF08C
:1058E00012008984000EC76E220EC66E9E96C69E5A
:1058F000870EC96EFF0E9EB602D0E82EFCD79E968C
:10590000C69EABC5C9FFFF0E9EB602D0E82EFCD7DF
:105910009E96C69EACC5C9FFFF0E9EB602D0E82E6D
:10592000FCD79E96C69EADC5C9FFFF0E9EB602D09F
:10593000E82EFCD79E96C69EAEC5C9FFFF0E9EB64A
:1059400002D0E82EFCD789941AEC2EF089849E961A
:10595000C69E8F0EC96EFF0E9EB602D0E82EFCD7F3
:105960009E96C69EB3C5C9FFFF0E9EB602D0E82E16
:10597000FCD789941AEC2EF012008984000EC76EB1
:10598000220EC66E9E96C69E870EC96EFF0E9EB6EE
:1059900002D0E82EFCD79E96C69E000EC96EFF0E62
:1059A0009EB602D0E82EFCD79E96C69E800EC96E8B
:1059B000FF0E9EB602D0E82EFCD79E96C69E800EA5
:1059C000C96EFF0E9EB602D0E82EFCD79E96C69EEC
:1059D000800EC96EFF0E9EB602D0E82EFCD78994C9
:1059E0001AEC2EF089849E96C69E8F0EC96EFF0E0D
:1059F0009EB602D0E82EFCD79E96C69E010EC96EBA
:105A0000FF0E9EB602D0E82EFCD789941AEC2EF039
:105A100012008984000EC76E220EC66E9E96C69E28
:105A2000870EC96EFF0E9EB602D0E82EFCD79E965A
:105A3000C69E000EC96EFF0E9EB602D0E82EFCD7A1
:105A40009E96C69E000EC96EFF0E9EB602D0E82E30
:105A5000FCD79E96C69E800EC96EFF0E9EB602D0E3
:105A6000E82EFCD79E96C69E800EC96EFF0E9EB68F
:105A700002D0E82EFCD789941AEC2EF089849E96E9
:105A8000C69E8F0EC96EFF0E9EB602D0E82EFCD7C2
:105A90009E96C69E010EC96EFF0E9EB602D0E82EDF
:105AA000FCD789941AEC2EF012008984000EC76E80
:105AB000220EC66E9E96C69E8F0EC96EFF0E9EB6B5
:105AC00002D0E82EFCD71AEC2EF09E96C69E810ED0
:105AD000C96EFF0E9EB602D0E82EFCD789941AEC50
:105AE0002EF08984000EC76E220EC66E9E96C69E4C
:105AF0008F0EC96EFF0E9EB602D0E82EFCD71AECB0
:105B00002EF09E96C69E010EC96EFF0E9EB602D066
:105B1000E82EFCD789941AEC2EF089849E96C69EB6
:105B2000910EC96EFF0E9EB602D0E82EFCD71AEC7D
:105B30002EF09E96C69EA50EC96EFF0E9EB602D092
:105B4000E82EFCD789941AEC2EF012008984000EFE
:105B5000C76E220EC66E9E96C69E8F0EC96EFF0E33
:105B60009EB602D0E82EFCD71AEC2EF09E96C69E6A
:105B7000810EC96EFF0E9EB602D0E82EFCD7899426
:105B80001AEC2EF012008984000EC76E220EC66E2B
:105B90009E96C69E8F0EC96EFF0E9EB602D0E82E50
:105BA000FCD71AEC2EF09E96C69E010EC96EFF0E13
:105BB0009EB602D0E82EFCD789941AEC2EF0120083
:105BC0008984000EC76E220EC66E9E96C69E910EEA
:105BD000C96EFF0E9EB602D0E82EFCD71AEC2EF04E
:105BE0009E96C69EA50EC96EFF0E9EB602D0E82EEA
:105BF000FCD789941AEC2EF012008984000EC76E2F
:105C0000220EC66E9E96C69E910EC96EFF0E9EB661
:105C100002D0E82EFCD71AEC2EF09E96C69E000EFF
:105C2000C96EFF0E9EB602D0E82EFCD789941AECFE
:105C30002EF01200050EE82EFED712000501256B8E
:105C4000266B276B286B899A400EC76E200EC66E96
:105C50009E96C69E030EC96EFF0E9EB602D0E82E1B
:105C6000FCD79E96C69E27C5C9FFFF0E9EB602D0E2
:105C7000E82EFCD79E96C69E26C5C9FFFF0E9EB68F
:105C800002D0E82EFCD79E96C69E25C5C9FFFF0E02
:105C90009EB602D0E82EFCD79E96C69EC952FF0E35
:105CA0009EB602D0E82EFCD7898A0F01C950FF0AA0
:105CB00001E1120005012E51130A05E005012E51E4
:105CC000170A0CE012000501E00E256FFF0E266F8B
:105CD0000F0E276F000E286F77EF2EF00501E00EF4
:105CE000256FFF0E266FFF0E276F000E286F899A13
:105CF000400EC76E200EC66E9E96C69E030EC96EDF
:105D0000FF0E9EB602D0E82EFCD79E96C69E27C5F3
:105D1000C9FFFF0E9EB602D0E82EFCD79E96C69E07
:105D200026C5C9FFFF0E9EB602D0E82EFCD79E9670
:105D3000C69E25C5C9FFFF0E9EB602D0E82EFCD731
:105D40009E96C69EC952FF0E9EB602D0E82EFCD784
:105D5000898A0F01C950FF0A1DE005012E51130A5F
:105D600005E005012E51170A0BE012000501000E97
:105D7000256F000E266F100E276F000E286F120081
:105D80000501000E256F000E266F000E276F010E15
:105D9000286F12000501256B266B276B286B050108
:105DA0002E51130A05E005012E51170A0CE01200CE
:105DB0000501000E216F000E226F040E236F000EEE
:105DC000246FECEF2EF00501000E216F000E226F04
:105DD000800E236F000E246F21C500F122C501F152
:105DE00023C502F124C503F125C504F126C505F13B
:105DF00027C506F128C507F124EC27F000C125F5D9
:105E000001C126F502C127F503C128F5899A400E84
:105E1000C76E200EC66E9E96C69E030EC96EFF0EFE
:105E20009EB602D0E82EFCD79E96C69E27C5C9FF17
:105E3000FF0E9EB602D0E82EFCD79E96C69E26C5C3
:105E4000C9FFFF0E9EB602D0E82EFCD79E96C69ED6
:105E500025C5C9FFFF0E9EB602D0E82EFCD79E9640
:105E6000C69EC952FF0E9EB602D0E82EFCD7898A84
:105E7000C950FF0A08E104C125F505C126F506C190
:105E800027F507C128F5D8900501243323332233A1
:105E900021332151E00B216F216756EF2FF022674C
:105EA00056EF2FF0236756EF2FF02467ECEF2EF01C
:105EB0000501200E2527E86A2623E86A2723E86AD9
:105EC00028231200E86A05012E51130A06E0050195
:105ED0002E51170A0BE0020E120005012851000A8C
:105EE00003E12751F00B07E0010E120005012851D4
:105EF000000A01E0010E120029C500F12AC501F1D6
:105F00002BC502F12CC503F125C504F126C505F109
:105F100027C506F128C507F1B3EC28F003BF12002E
:105F200062EC2FF05FE1899A400EC76E200EC66EBC
:105F30009E96C69E060EC96EFF0E9EB602D0E82E35
:105F4000FCD7898A899A9E96C69E020EC96EFF0E5C
:105F50009EB602D0E82EFCD79E96C69E27C5C9FFE6
:105F6000FF0E9EB602D0E82EFCD79E96C69E26C592
:105F7000C9FFFF0E9EB602D0E82EFCD79E96C69EA5
:105F800025C5C9FFFF0E9EB602D0E82EFCD79E960F
:105F9000C69E000EC96EFF0E9EB602D0E82EFCD73C
:105FA000898A899A9E96C69E050EC96EFF0E9EB678
:105FB00002D0E82EFCD79E96C69EC952FF0E9EB612
:105FC00002D0E82EFCD7C9B0DBEF2FF0898A05019B
:105FD000200E2527E86A2623E86A2723E86A282373
:105FE0007CEF2FF01200899A400EC76E200EC66E0D
:105FF0009E96C69E060EC96EFF0E9EB602D0E82E75
:10600000FCD7898A899A9E96C69EC70EC96EFF0ED6
:106010009EB602D0E82EFCD7898A0501256B266B37
:10602000276B286B1200899A400EC76E200EC66E31
:106030009E96C69E050EC96EFF0E9EB602D0E82E35
:10604000FCD79E96C69EC952FF0E9EB602D0E82E81
:10605000FCD7C9CF33F5898A1200899A400EC76EE2
:10606000200EC66E9E96C69EB90EC96EFF0E9EB6D7
:1060700002D0E82EFCD7898A1200899A400EC76E9A
:10608000200EC66E9E96C69EAB0EC96EFF0E9EB6C5
:1060900002D0E82EFCD7898AFF0EE82EFED7120028
:1060A00062EC2FF0D8A41200899A400EC76E200E21
:1060B000C66E9E96C69E030EC96EFF0E9EB602D099
:1060C000E82EFCD79E96C69E27C5C9FFFF0E9EB63A
:1060D00002D0E82EFCD79E96C69E26C5C9FFFF0EAD
:1060E0009EB602D0E82EFCD79E96C69E25C5C9FF57
:1060F000FF0E9EB602D0E82EFCD79E96C69EC952D1
:10610000FF0E9EB602D0E82EFCD7898A0F01C95037
:10611000FF0AD8A445EF33F00501FE0E336F67EC9C
:106120002BF0ABC534F5ACC535F5ADC536F5AEC510
:1061300037F5AFC538F5B0C539F5B1C53AF50784BF
:10614000B6C166F1B7C167F1B8C168F1B9C169F10B
:106150004BC14FF14CC150F14DC151F14EC152F103
:1061600057C159F158C15AF138EC1EF000C13BF546
:1061700001C13CF502C13DF503C13EF505015D6776
:10618000C9EF30F05E67C9EF30F05F67C9EF30F0FC
:106190006067CDEF30F0DAEF30F05DC504F15EC539
:1061A00005F15FC506F160C507F1B3EC28F003BF48
:1061B00045EF33F059C13FF55AC140F5B5C541F53A
:1061C000B6C542F52BEC26F036C645F537C646F582
:1061D00006014067F3EF30F04167F3EF30F04267BC
:1061E000F3EF30F04367F7EF30F008EF31F0AEEC4B
:1061F00029F0B4EC29F036C600F137C601F140C6EB
:1062000004F141C605F1B3EC28F003AF45EF33F0DC
:106210000101036B026B1AC600F11BC601F101AF4D
:1062200016EF31F0FF0E026FFF0E036F0101076BD7
:10623000066B1CC604F11DC605F105AF24EF31F055
:10624000FF0E066FFF0E076FB8EC28F00101076B19
:10625000066B1EC604F11FC605F105AF34EF31F021
:10626000FF0E066FFF0E076FB8EC28F00101076BF9
:10627000066B20C604F121C605F105AF44EF31F0ED
:10628000FF0E066FFF0E076FB8EC28F0D8900101E3
:106290000333023301330033D89001010333023357
:1062A0000133003300C147F501C148F50101036B1B
:1062B000026B22C600F123C601F101AF64EF31F099
:1062C000FF0E026FFF0E036F0101076B066B24C602
:1062D00004F125C605F105AF72EF31F0FF0E066F30
:1062E000FF0E076FB8EC28F00101076B066B26C69E
:1062F00004F127C605F105AF82EF31F0FF0E066FFE
:10630000FF0E076FB8EC28F00101076B066B28C67B
:1063100004F129C605F105AF92EF31F0FF0E066FCB
:10632000FF0E076FB8EC28F0D89001010333023359
:1063300001330033D89001010333023301330033BA
:1063400000C149F501C14AF50101036B026B2AC680
:1063500000F12BC601F101AFB2EF31F0FF0E026F79
:10636000FF0E036F0101076B066B2CC604F12DC6EF
:1063700005F105AFC0EF31F0FF0E066FFF0E076F9E
:10638000B8EC28F00101076B066B2EC604F12FC68E
:1063900005F105AFD0EF31F0FF0E066FFF0E076F6E
:1063A000B8EC28F00101076B066B30C604F131C66A
:1063B00005F105AFE0EF31F0FF0E066FFF0E076F3E
:1063C000B8EC28F0D89001010333023301330033D5
:1063D000D8900101033302330133003300C14BF580
:1063E00001C14CF50101036B026B02C600F103C64B
:1063F00001F101AF00EF32F0FF0E026FFF0E036FED
:106400000101076B066B04C604F105C605F105AF73
:106410000EEF32F0FF0E066FFF0E076FB8EC28F09C
:106420000101076B066B06C604F107C605F105AF4F
:106430001EEF32F0FF0E066FFF0E076FB8EC28F06C
:106440000101076B066B08C604F109C605F105AF2B
:106450002EEF32F0FF0E066FFF0E076FB8EC28F03C
:10646000D89001010333023301330033D890010186
:10647000033302330133003300C14DF501C14EF542
:106480000101036B026B0AC600F10BC601F101AFFB
:106490004EEF32F0FF0E026FFF0E036F0101076B2C
:1064A000066B0CC604F10DC605F105AF5CEF32F0CA
:1064B000FF0E066FFF0E076FB8EC28F00101076BA7
:1064C000066B0EC604F10FC605F105AF6CEF32F096
:1064D000FF0E066FFF0E076FB8EC28F00101076B87
:1064E000066B10C604F111C605F105AF7CEF32F062
:1064F000FF0E066FFF0E076FB8EC28F0D890010171
:106500000333023301330033D890010103330233E4
:106510000133003300C14FF501C150F50101036B98
:10652000026B12C600F113C601F101AF9CEF32F00D
:10653000FF0E026FFF0E036F0101076B066B14C69F
:1065400004F115C605F105AFAAEF32F0FF0E066F94
:10655000FF0E076FB8EC28F00101076B066B16C63B
:1065600004F117C605F105AFBAEF32F0FF0E066F62
:10657000FF0E076FB8EC28F00101076B066B18C619
:1065800004F119C605F105AFCAEF32F0FF0E066F30
:10659000FF0E076FB8EC28F0D890010103330233E7
:1065A00001330033D8900101033302330133003348
:1065B00000C151F501C152F507940501200E326F5B
:1065C000899A400EC76E200EC66E9E96C69E060E17
:1065D000C96EFF0E9EB602D0E82EFCD7898A899A32
:1065E0009E96C69E020EC96EFF0E9EB602D0E82E83
:1065F000FCD79E96C69E27C5C9FFFF0E9EB602D049
:10660000E82EFCD79E96C69E26C5C9FFFF0E9EB6F5
:1066100002D0E82EFCD79E96C69E25C5C9FFFF0E68
:106620009EB602D0E82EFCD725EE33F0322F02D0F2
:1066300025EF33F09E96C69EDECFC9FFFF0E9EB6B5
:1066400002D0E82EFCD716EF33F0898A899A9E96FD
:10665000C69E050EC96EFF0E9EB602D0E82EFCD770
:106660009E96C69EC952FF0E9EB602D0E82EFCD75B
:10667000C9B030EF33F0898A0501200E2527E86A7A
:106680002623E86A2723E86A2823120021C500F19F
:1066900022C501F123C502F124C503F1899A400EF8
:1066A000C76E200EC66E9E96C69E0B0EC96EFF0E5E
:1066B0009EB602D0E82EFCD79E96C69E02C1C9FFA8
:1066C000FF0E9EB602D0E82EFCD79E96C69E01C154
:1066D000C9FFFF0E9EB602D0E82EFCD79E96C69E3E
:1066E00000C1C9FFFF0E9EB602D0E82EFCD79E96D1
:1066F000C69EC952FF0E9EB602D0E82EFCD725EEEC
:1067000033F00501200E326F9E96C69EC952FF0ED1
:106710009EB602D0E82EFCD7C9CFDEFF322F84EF21
:1067200033F0898A1200899A400EC76E200EC66E19
:106730009E96C69E900EC96EFF0E9EB602D0E82EA3
:10674000FCD79E96C69E000EC96EFF0E9EB602D066
:10675000E82EFCD79E96C69E000EC96EFF0E9EB612
:1067600002D0E82EFCD79E96C69E000EC96EFF0E84
:106770009EB602D0E82EFCD79E96C69EC952FF0E4A
:106780009EB602D0E82EFCD7C9CF2DF59E96C69EA8
:10679000C952FF0E9EB602D0E82EFCD7C9CF2EF507
:1067A000898A12009FEC27F0B5C5E8FFD70802E3FD
:1067B0009FEC27F0B5C5E8FFC80802E39FEC27F07F
:1067C000B5C5E8FFB90802E39FEC27F0B5C5E8FFBF
:1067D000AA0802E39FEC27F0B5C5E8FF9B0802E397
:1067E0009FEC27F017EC2CF02DEC30F0F29CF29E91
:1067F0008B94C69AC290898C9482948C720ED36EBC
:10680000D3A4FED789968A909390FF0EE8CF00F02C
:10681000E82EFED7002EFCD78150F294F29A9E907B
:106820009D909E929D92F298F292F290F286F28E54
:046830000300FF0062
:10BF0000E844F926000C160C2B0C3F0C520C640C68
:10BF1000760C860C960CA50CB30CC10CCF0CDC0C6B
:06BF2000E80CF40C000C1B
:00000001FF
